:1000000075817F7401F58F538EF1438E10C2D4C277
:04001000D3020036E1
:0300230002AA6DC1
:03002B0002AAA87E
:1000330002AA3EC204753E00753F00D291C2B7C208
:10004300B6C2B57550FF7551FFD2A1D2B2D2B3C2B9
:10005300167541FF75427FC217C218C219C21AC270
:100063001BC21CC21DC21EC21FC220C221C222D279
:1000730023D224D225D226D227D228D229D22AD2B9
:100083002BD22CD22DD22EC253C252D252C232C242
:1000930055C256D233D247C236C237C257C258C2EC
:1000A3005DC25CC238C239C20CC24CD23AD23BC226
:1000B3003C756C00756D00756F00756E0075717F12
:1000C30075707FC249C24AD24BD24DC24E7567008A
:1000D300756800C209C20EC20BD20DC20F7544006F
:1000E30075450075460075470075480075490075EC
:1000F3004A00754B00754C00754D00754E00754FE9
:1001030000D212D213755B00755C00755D00755EDD
:100113000075610075620075630075640075730690
:1001230075740075760675770075431875790175D2
:100133007A01740090003FF0900040F0743E90000C
:1001430041F07400900072F0900073F0900074F02E
:10015300900075F0900076F07401900177F09001B3
:1001630078F0900179F07400900176F090017AF0C4
:10017300740190017EF090017CF090017DF090017C
:1001830084F090017FF0900180F0900181F0900164
:1001930082F0900183F0900186F0900185F0900148
:1001A30088F0129D489001D87400F074F090019883
:1001B300F0749F900199F074C39001AFF0740390B1
:1001C30001B0F09006F57400F07417900077F074A6
:1001D30005900078F0740F900079F0740190018716
:1001E300F0129D94129D79129D82129D8B129DB2E5
:1001F300129DCC129D29740090021DF07400900290
:10020300B6F0129D3574009004D2F0740090056B23
:10021300F0740C79FF9002B7F0A3F0D9FC740C7959
:10022300FF9003B7F0A3F0D9FC74009004B7F07407
:10023300009004B8F0740C79FF90056CF0A3F0D92A
:10024300FC740090066CF0740090066DF0740090DE
:1002530006D7F074009006E1F09006E2F09006E312
:10026300F09006E4F09006E5F09006E6F09006E7DD
:10027300F09006EA7400F0126C15126C4A7550FF88
:100283007551FF12845D75520012971F12903F75CE
:100293003D0012AA2112A9DF5350DF12921D1293BF
:1002A300BA7550FF7551FF12919E1294D61294E6BF
:1002B300900200E0F569123122123BAE7402900104
:1002C3007DF0124DFD740390017DF0124DFD740419
:1002D30090017DF0124DFD740590017DF0124DFDEE
:1002E300740690017DF0124DFD740790017DF012AC
:1002F3004DFD740890017DF0124DFD740190017D58
:10030300F0124DFD9001FEE0A2E2925912457412E3
:1003130094999001F9E09006E8F09001FAE09006D4
:10032300E9F0122C59122EDE122E89128E2712A9F1
:1003330075539EE29006A57400F0C203C202121028
:10034300C4020341783279FF0000D9FCD8F822783F
:100353004B79FF0000D9FCD8F82278327932D9FEE4
:10036300D8FA22F87902D9F6D8F222E627F52C0832
:1003730009E637F52D782C22C3E697F52C0809E614
:1003830097F52D782C22862C872E0809862D872F0A
:1003930012040E78312286310886320886330886A5
:0B03A30034872E09872F1203B1782C3D
:1003AE007933227535007536101203F31203C41219
:1003BE0003E7D536F422C3E533952EE534952FE5C4
:1003CE00359400500122E533952EF533E534952F03
:1003DE00F534E5359400F53522B3E52C33F52CE5EF
:1003EE002D33F52D22C3E53133F531E53233F532B8
:1003FE00E53333F533E53433F534E53533F535226E
:10040E00E52C852EF0A4F53185F032E52D852FF003
:10041E00A4F53385F034E52D852EF0A42532F53282
:10042E00E53335F0F533E5343400F534E52C852F1E
:10043E00F0A42532F532E53335F0F533E5343400EA
:10044E00F53422E582C4540FF9E583C46922E582AE
:10045E000303543FF9E583030354C069227A0CC2A7
:10046E0097D2A3A29633C933C9C2A3DAF2F8D297B0
:10047E0022C2A3C2973392A6D2A3DAF5C2A3120464
:10048E006BE95403F9227A0574E012047FF5838830
:10049E0082227A0574D812047FF5838882227A0527
:1004AE0074C012047FF5838882227A0574C8120400
:1004BE007FF5838882227A0574D012047FF58388B3
:1004CE0082227A0574E812047FF5838882227A05E7
:1004DE0074F012047FF5838882227A0574F8120470
:1004EE007FF583888222C2B41205041205511205CB
:1004FE009ED2B4C2B422A846A947E9540F44507AFA
:10050E0008C2A1C2A33392A6D2A3DAF77A08E8C230
:10051E00A33392A6D2A3DAF7C2A3D2A1A844A945C7
:10052E00E9540F44D07A08C2A1C2A33392A6D2A333
:10053E00DAF77A08E8C2A33392A6D2A3DAF7C2A3F7
:10054E00D2A122A84AA94BE9540F44507A08C2B24C
:10055E00C2A33392A6D2A3DAF77A08E8C2A33392E3
:10056E00A6D2A3DAF7C2A3D2B2A84EA94FE9540F6E
:10057E0044D07A08C2B2C2A33392A6D2A3DAF77AD3
:10058E0008E8C2A33392A6D2A3DAF7C2A3D2B2224C
:10059E00A848A949E9540F44507A08C2B3C2A333FC
:1005AE0092A6D2A3DAF77A08E8C2A33392A6D2A310
:1005BE00DAF7C2A3D2B3A84CA94DE9540F44D07AAE
:1005CE0008C2B3C2A33392A6D2A3DAF77A08E8C25E
:1005DE00A33392A6D2A3DAF7C2A3D2B322F537750C
:1005EE0038007837753B22753C00793B12038986BB
:1005FE008208868322F5377538007837753B447547
:10060E003C00793B120389868208868322F5377572
:10061E0038007837753B20753C00793B120389868C
:10062E00820886832220A204753E002220A003D2D7
:10063E000422753E0122E53EB53F04853E3F22B4BD
:10064E00001520040A0540853E3FD206D20222C282
:10065E0004853E3FD2062220040A1540853E3FD235
:10066E0006D20322C204853E3FD20622E56B20E667
:10067E0001229006EAE0700302069E0206E7E56B91
:10068E0020E601229006EAE07003020730020779A5
:10069E009006EBE01475F006A49006AB73900198EB
:1006AE000207C29001980207C29001980207E890D3
:1006BE0001980207F89001980207C290019802076C
:1006CE00C29001980207C29001980207C290019849
:1006DE000207C29001980207C29006EBE01475F073
:1006EE0006A49006F4739001990207C29001990234
:1006FE0007DB90019902084C90019902084C900179
:10070E009902080E90019902081290019902081997
:0E071E009001990207E89001990208239001CA
:10072C00990208369006ECE01475F006A490073D8B
:10073C00739001AF0207C29001AF0207C29001AFE4
:10074C000207E89001AF0207F89001AF0207C290D0
:10075C0001AF0207C29001AF0207C29001AF0207BE
:10076C00C29001AF0207C29001AF0207C29006EC23
:10077C00E01475F006A4900786739001B00207C2CE
:10078C009001B00207DB9001B002084C9001B0025E
:10079C00084C9001B002080E9001B00208129001B2
:1007AC00B00208199001B00207E89001B0020823CA
:1007BC009001B002083612084D12086612087F121A
:1007CC0008981208B11208CA1208E31208FC221287
:1007DC00084D12086612087F1208982212084D1252
:1007EC00086612087F1208981208B12212084D12DE
:1007FC00086612087F1208981208B11208CA12086B
:10080C00E32212084D2212084D1208662212084DDE
:10081C0012086612087F2212084D12086612087F11
:10082C001208981208B11208CA2212084D12086652
:10083C0012087F1208981208B11208CA1208E32293
:10084C0022E56B30E108C21720230ED22322C223EB
:10085C00201706D217E0B2E7F022E56B30E208C2AF
:10086C001820240ED22422C224201806D218E0B25A
:10087C00E6F022E56B30E308C21920250ED22522C2
:10088C00C225201906D219E0B2E5F022E56A30E162
:10089C0008C21A20260ED22622C226201A06D21AE6
:1008AC00E0B2E4F022E56A30E208C21B20270ED247
:1008BC002722C227201B06D21BE0B2E3F022E56AF6
:1008CC0030E308C21C20280ED22822C228201C0685
:1008DC00D21CE0B2E2F022E56A30E508C21D202904
:1008EC000ED22922C229201D06D21DE0B2E1F0222F
:1008FC00E56A30E708C21E202A0ED22A22C22A201C
:10090C001E06D21EE0B2E0F022E56A30E40630E6C4
:10091C0011C2382230380122D2389006EAE0740035
:10092C00F02230380122D2389006EAE07401F0222D
:10093C009006EAE07009E551C2E3D2E5F55122E5F3
:10094C0051D2E3C2E5F55122120A1B9006EAE0707F
:10095C0007900198120982229001991209822212A1
:10096C000A1B9006EAE070079001AF1209822290F0
:10097C0001B012098222E020E709E550D2E1F550DE
:10098C00020995E550C2E1F550E020E609E550D2A8
:10099C00E2F5500209A8E550C2E2F550E020E50965
:1009AC00E550D2E3F5500209BBE550C2E3F550E047
:1009BC0020E409E550D2E6F5500209CEE550C2E636
:1009CC00F550E020E309E550D2E7F5500209E1E5E6
:1009DC0050C2E7F550E020E209E551D2E1F55102B1
:1009EC0009F4E551C2E1F551E020E109E551D2E409
:1009FC00F551020A07E551C2E4F551E020E009E5A2
:100A0C0051D2E7F551020A1AE551C2E7F55122E538
:100A1C0050D2E4F550E551D2E0D2E2D2E6F55122C3
:100A2C00B4FF03740022B4EB012250012274EB22B8
:100A3C00B4FF03740022B40F0122500122740F2260
:100A4C00B40101225003740122B4EC0122500122A2
:100A5C0074EC22B4FF03740022B40C012250012266
:100A6C00740C22B40101225003740122B41001222F
:100A7C00500122741022B40101225003740122B4DB
:100A8C000A0122500122740A22B40101225003747B
:0E0A9C000122B4200122500122742022B40154
:100AAA0001225003740122B41F0122500122741F33
:100ABA0022B40101225003740122B4080122500118
:100ACA0022740822B40101225003740122B41101D4
:100ADA0022500122741122B401012250037401220E
:100AEA00B47F0122500122747F22B4FF03740022D2
:100AFA00B4030122500122740322B4EB01225001F3
:100B0A002274EB22B40101225003740122B40A01B7
:100B1A0022500122740A22B40101225003740122D4
:100B2A00B40C0122500122740C22B4010122500398
:100B3A00740122B4030122500122740322B4010178
:100B4A00225003740122B40901225001227409229D
:100B5A00B40101225003740122B40301225001227C
:100B6A00740322B40101225003740122B405012244
:100B7A00500122740522B40101225003740122B4E7
:100B8A00030122500122740322B40101225003748A
:100B9A000122B4030122500122740322B40101226A
:100BAA005003740122B4060122500122740622B4B1
:100BBA000101225003740122B41901225001227446
:100BCA001922B40101225003740122B422012250D5
:100BDA000122742222B40101225003740122B40AB0
:100BEA000122500122740A22B40101225003740125
:100BFA0022B4070122500122740722B4FF037400B1
:100C0A0022B47E0122500122747E22B403012250B2
:100C1A0003740322B48F0122500122748F22B4017B
:100C2A0001225003740122B40401225001227404E7
:100C3A0022B40101225003740122B402012250019C
:100C4A0022740222B40101225003740122B4020167
:100C5A0022500122740222B401012250037401229B
:100C6A00B4020122500122740222B401012250036B
:100C7A00740122B4030122500122740322B4010137
:100C8A00225003740122B45F0122500122745F22B0
:100C9A00B4FF08B9000374FE22740022B4010122D1
:100CAA005003740122B4110122500122741122B49A
:100CBA000101225003740122B40501225001227459
:100CCA000522B40101225003740122B40B012250FF
:100CDA000122740B22B40101225003740122B57C53
:100CEA000122500122E57C22B40101225003740141
:100CFA0022B43A0122500122743A22B4010122504C
:100D0A0003740122B4460122500122744622B4011E
:100D1A0001225003740122B48001225001227480FE
:100D2A0022B40101225003740122B40701225001A6
:100D3A0022740722B40101225003740122B40C0167
:100D4A0022500122740C22B40101225003740122A0
:100D5A00B40C0122500122740C22B4010122500366
:100D6A00740122B40C0122500122740C22B4010134
:100D7A00225003740122B41701225001227417224F
:100D8A00300909C209300A02C20AD20B229006A50A
:100D9A00E020E4012230E607C2E4C2E6F0D25E2295
:100DAA00121348120D97305E09C25E300A02C20A57
:100DBA00D20B22304F15E56B30E61030E003C20C3F
:100DCA0022200C07D20CB20E120DD622300E0AD2F5
:100DDA000AD20ED20F5350DF22D20DC20EC20B43DB
:100DEA00502022900189E02414FA74003400FB7523
:100DFA0037D0753812753913753A0078378A3B8BB4
:100E0A003C793B120399E6F54108E6F54222D211F4
:0E0E1A00F5992011FD22B4F808300A02C20A30
:100E2800D20B22B4FA0AD20AD20ED20F5350DF22C2
:100E3800B4FC0AD20DC20EC20B43502022B4FB09E7
:100E4800D20AD20ED20F5350DF22B4F007756700D2
:100E580075680022B4F10775670075680022B4F25E
:100E68000775670075680022B4F30F756700756829
:100E78000022304F0122120E202250F6E5692490FC
:100E8800F57EE9B57E08756701C250C25422E5694E
:100E98002480F57EE9B57E08756801D250C25422D7
:100EA800E56924B0F57EE9B57E06756701D254225E
:100EB80030E70D75670075680022020F07020F1DE5
:100EC8002054FA2050F4A967B9000122A967B90192
:100ED800050567F56522B9021405676008E565121E
:100EE8001012D24E22E565121057D24E22B90305D0
:100EF8000567F56522B90406756701020EE322A9A4
:100F080068B9000122A968B901070568F565020EEC
:100F1800ED75680122A967B9000122A967B9010521
:100F28000567F57F22B902090567F9120F4BD24E02
:100F380022B903050567F57F22B904067567010222
:100F48000F3222E57FB41403020F5D500122B41E54
:100F58000122400122C3941475F003A4900F687312
:100F6800020F86020F8F020F9D020FAD020FBC0207
:100F78000FCC020FD5020FE3020FF3021002E912A1
:100F88000C0590018DF022E975F00C8404120CCC4C
:100F9800900190F022E975F00E8404120BDF9001A5
:100FA8008BF0D23222E975F00584120BB990018AD0
:100FB800F0D23222E975F00F8404120CB990018C3A
:100FC800F0D23222E9120C059001A4F022E975F062
:100FD8000C8404120CCC9001A7F022E975F00E8461
:100FE80004120BDF9001A2F0D23222E975F00584D9
:100FF800120BB99001A1F0D23222E975F00F8404E6
:10100800120CB99001A3F0D23222B42426C3940C56
:10101800FE9418FF90022A1210A0E0D2E7F0128E78
:1010280032EEFF9004DF1210BEE0D2E7F0128EE439
:10103800D2322250D8B40B012240FDC3940CFF9049
:1010480004DF1210BEE0D2E7F0128EE4D232223072
:101058003A0122B42426C3940CFE9418FF90022A65
:101068001210A0E0C2E7F0128E4AEEFF9004DF12E1
:1010780010BEE0C2E7F0128EFCD2322250D8B40B78
:10108800012240FDC3940CFF9004DF1210BEE0C2A1
:10109800E7F0128EFCD23222128C96EF240C858255
:1010A800378583387837F53B753C00793B12036EFA
:1010B800868208868322128CA40210A312A0BE1274
:1010C800A0F112A4F712A8E412A9471237C4128D8E
:1010D80004128D881284B912973B129B8B1250AB65
:1010E800128B2E90017CE0B4060A900183E0B403D1
:1010F800030210FF12999F126C15122AA09001FD8D
:10110800E0B4040302111202118D121311121372AA
:101118009006A5E020E205D29102113330E50CC219
:10112800911213A79006A5E0C2E5F09006A5E0206D
:10113800E40612284E02115030E60D12181C12282F
:101148007F9006A5E0C2E6F09006A5E020E0081230
:1011580022FFC2B602116F30E10D1217F212206F92
:101168009006A5E0C2E1F09006A5E020E30612256E
:10117800FEC2B52230E70D12180712236E9006A59D
:10118800E0C2E7F022120DBD304F139001FDE0B42C
:0E1198000306120DAA0211A6120DED120D8A09
:1011A600126C15200D030211C8C20D9001FCE0B4AB
:1011B60001030211C074FC120E181212C0C2B7123B
:1011C6009A2A300F11C20F9001FCE0B401030211FC
:1011D600DC74FA120E18300A05D2480210C4200E2A
:1011E60003021239200B03021239C20B9001FCE0F4
:1011F600B40103021211B4020874F8120E18021296
:1012060011B25B305B0574F8120E18204F0B305983
:1012160008B25A305A0302123930480B12123AC237
:1012260048129DB202123912202012231D1213D920
:10123600121270221212C0C24B128B5D125D1190F7
:1012460004B8E0149004B7F01264CF90066DE01471
:1012560090066CF0E550C2E5F550D2B712200D129B
:1012660099E2121270C249C24A22122069122173EF
:1012760012236812247212261C7E011226DD122702
:101286008D7E021226DD12278D7E031226DD1227A1
:101296008D7E041226DD12278D7E051226DD12278D
:1012A6008D7E061226DD12278D7E071226DD122779
:1012B6008D7E081226DD12278D22435020122191A1
:1012C6001224907400900077F090014BF090014D3D
:1012D600F090014EF0900150F0755200129D791277
:1012E6009D82129D8B129DB2129F4D90019EE0141D
:1012F600A3F0129F989001B5E014A3F0C255C25610
:101306009001757400F0C25AC25B2212131E1213AA
:101316003312134812135D222090089006A5E0D2DE
:10132600E0F0229006A5E0C2E0D2E1F02220930888
:101336009006A5E0D2E3F0229006A5E0C2E3D2E74C
:10134600F0222094089006A5E0D2E4F0229006A5AB
:10135600E0C2E4D2E6F0222092089006A5E0D2E2AE
:10136600F0229006A5E0C2E2D2E5F022E56B30E677
:101376002F30E003C20C22200C26D20C1213A71227
:1013860022FF1225FE1229A81229C71229E6122ABF
:1013960005122A24122A43122A62122A81129A2A32
:1013A600229004B8E0149004B7F090066DE0149013
:1013B600066CF074FF90014BF090014DF090014ED9
:1013C600F0900150F074FF129D7B74FF129D841201
:1013D6009DB7221217F212183112184B12187912F1
:1013E60018931218AD1218C71218E1121901121922
:1013F6001B12193512194F12196912198312199DE8
:101406001219B71219D122E01475F004A49014171A
:1014160073EF0214F0EF0216BEEF02153DEF021550
:101426008AEF0215D7EF021624EF021671EF0217A4
:101436000BEF021758EF0217A5E01475F004A490FD
:1014460014497390007D22900110229000B12290E1
:1014560000C4229000D7229000EA229000FD22903C
:101466000123229001362290014922E01475F004EE
:10147600A490147B7390007F22900111229000B2F9
:10148600229000C5229000D8229000EB229000FE08
:1014960022900124229001372290014A221475F0ED
:1014A60004A49014AC7390007A22900082229000DB
:1014B600862290008C229000922290009822900022
:1014C6009E22900080229000842290008822900024
:1014D6008E229000942290009A2290008A229000F8
:1014E60090229000962290009C221475F004A490FD
:1014F60014F97390007B229000832290008722903B
:10150600008D22900093229000992290009F2290B5
:0E151600008122900085229000892290008F93
:10152400229000952290009B2290008B22900091A3
:10153400229000972290009D221475F004A4901527
:1015440046739000A0229000A2229000A422900052
:10155400A7229000AA229000AD229000B022900011
:10156400A1229000A3229000A5229000A82290001E
:10157400AB229000AE229000A6229000A9229000F7
:10158400AC229000AF221475F004A49015937390CC
:1015940000B3229000B5229000B7229000BA2290A6
:1015A40000BD229000C0229000C3229000B422907B
:1015B40000B6229000B8229000BB229000BE229078
:1015C40000C1229000B9229000BC229000BF22905A
:1015D40000C2221475F004A49015E0739000C62292
:1015E4009000C8229000CA229000CD229000D02200
:1015F4009000D3229000D6229000C7229000C922E6
:101604009000CB229000CE229000D1229000D422D0
:101614009000CC229000CF229000D2229000D522BC
:101624001475F004A490162D739000D9229000DB59
:10163400229000DD229000E0229000E3229000E658
:10164400229000E9229000DA229000DC229000DE51
:10165400229000E1229000E4229000E7229000DF33
:10166400229000E2229000E5229000E8221475F016
:1016740004A490167A739000EC229000EE2290005D
:10168400F0229000F3229000F6229000F9229000BC
:10169400FC229000ED229000EF229000F1229000B5
:1016A400F4229000F7229000FA229000F222900097
:1016B400F5229000F8229000FB221475F004A49007
:1016C40016C7739000FF229001012290010322901B
:1016D4000106229001092290010C2290010F229010
:1016E400010022900102229001042290010722901D
:1016F400010A2290010D22900105229001082290F6
:10170400010B2290010E221475F004A49017147397
:1017140090011222900114229001162290011922A4
:1017240090011C2290011F22900122229001132279
:10173400900115229001172290011A2290011D2276
:10174400900120229001182290011B2290011E2258
:10175400900121221475F004A4901761739001255F
:1017640022900127229001292290012C2290012FFE
:1017740022900132229001352290012622900128E4
:101784002290012A2290012D2290013022900133CF
:101794002290012B2290012E2290013122900134BB
:1017A400221475F004A49017AE73900138229001AE
:1017B4003A2290013C2290013F2290014222900162
:1017C4004522900148229001392290013B22900148
:1017D4003D22900140229001432290014622900133
:1017E4003E22900141229001442290014722900020
:1017F4007A7400F01219EE90007BE004B4100274C5
:1018040000F02290007C7400F0121A4090007DE0F9
:1018140004B410027400F02290007E7400F0121AD6
:101824009290007FE004B410027400F022900080D3
:10183400E004B402107400F0121AE4900081E00491
:10184400B410027400F022900082E004B403247403
:1018540000F0B2B7900194E0B40202C2B69001ABBA
:10186400E0B40202C2B5121B36900083E004B41047
:10187400027400F022900084E004B404107400F0B8
:10188400121B88900085E004B410027400F02290CA
:0E1894000086E004B406107400F0121BDA9017
:1018A2000087E004B410027400F022900088E00483
:1018B200B408107400F0121C2C900089E004B410DB
:1018C200027400F02290008AE004B409107400F05F
:1018D200121C7E90008BE004B410027400F022907F
:1018E200008CE004B40C167400F0E550B2E5F5503B
:1018F200121CD090008DE004B410027400F022900B
:10190200008EE004B410107400F0121D2290008FBB
:10191200E004B410027400F022900090E004B412CB
:10192200107400F0121D74900091E004B41002745F
:1019320000F022900092E004B418107400F0121D1E
:10194200C6900093E004B410027400F02290009458
:10195200E004B420107400F0121E18900095E00408
:10196200B410027400F022900096E004B4241074C3
:1019720000F0121E6A900097E004B410027400F0A6
:1019820022900098E004B430107400F0121EBC9053
:101992000099E004B410027400F02290009AE0046E
:1019A200B440107400F0121F0E90009BE004B410BB
:1019B200027400F02290009CE004B448107400F01D
:1019C200121F6090009DE004B410027400F0229097
:1019D200009EE004B460137400F012200D121FB2D6
:1019E20090009FE004B410027400F0229000A075F1
:1019F2007C051220049000B3757C0712200490002D
:101A0200C6757C091220049000D9757C0A12200444
:101A12009000EC757C0B1220049000FF757C0C1278
:101A22002004900112757C0D122004900125757C12
:101A32000E122004900138757C0F122004229000AF
:101A4200B1757C051220049000C4757C0712200435
:101A52009000D7757C091220049000EA757C0A1266
:101A620020049000FD757C0B122004900110757CFF
:101A72000C122004900123757C0D12200490013673
:101A8200757C0E122004900149757C0F12200422ED
:101A92009000B2757C051220049000C5757C071277
:101AA20020049000D8757C091220049000EB757C0C
:101AB2000A1220049000FE757C0B12200490011182
:101AC200757C0C122004900124757C0D1220049068
:101AD2000137757C0E12200490014A757C0F12208A
:101AE20004229000A1757C051220049000B4757C3C
:101AF200071220049000C7757C091220049000DAB6
:101B0200757C0A1220049000ED757C0B1220049063
:101B12000100757C0C122004900113757C0D1220BB
:101B220004900126757C0E122004900139757C0FF9
:101B3200122004229000A2757C051220049000B5A8
:101B4200757C071220049000C8757C09122004904D
:101B520000DB757C0A1220049000EE757C0B1220CB
:101B620004900101757C0C122004900114757C0D07
:101B7200122004900127757C0E12200490013A7500
:101B82007C0F122004229000A3757C051220049081
:101B920000B6757C071220049000C9757C091220DA
:101BA200049000DC757C0A1220049000EF757C0B17
:101BB200122004900102757C0C122004900115750C
:101BC2007C0D122004900128757C0E1220049001D5
:101BD2003B757C0F122004229000A4757C05122014
:101BE200049000B7757C071220049000CA757C0926
:101BF2001220049000DD757C0A1220049000F0751A
:101C02007C0B122004900103757C0C1220049001BD
:0E1C120016757C0D122004900129757C0E12AF
:101C2000200490013C757C0F122004229000A575C1
:101C30007C051220049000B8757C071220049000E7
:101C4000CB757C091220049000DE757C0A122004FA
:101C50009000F1757C0B122004900104757C0C122D
:101C60002004900117757C0D12200490012A757CC8
:101C70000E12200490013D757C0F1220042290006A
:101C8000A6757C051220049000B9757C071220040B
:101C90009000CC757C091220049000DF757C0A123C
:101CA00020049000F2757C0B122004900105757CD5
:101CB0000C122004900118757C0D12200490012B49
:101CC000757C0E12200490013E757C0F12200422B8
:101CD0009000A7757C051220049000BA757C07124D
:101CE00020049000CD757C091220049000E0757CE2
:101CF0000A1220049000F3757C0B12200490010658
:101D0000757C0C122004900119757C0D1220049032
:101D1000012C757C0E12200490013F757C0F12205F
:101D200004229000A8757C051220049000BB757CED
:101D3000071220049000CE757C091220049000E167
:101D4000757C0A1220049000F4757C0B122004901C
:101D50000107757C0C12200490011A757C0D12206D
:101D60000490012D757C0E122004900140757C0FAB
:101D7000122004229000A9757C051220049000BC5A
:101D8000757C071220049000CF757C091220049006
:101D900000E2757C0A1220049000F5757C0B12207D
:101DA00004900108757C0C12200490011B757C0DB9
:101DB00012200490012E757C0E12200490014175B2
:101DC0007C0F122004229000AA757C05122004903A
:101DD00000BD757C071220049000D0757C0912208C
:101DE000049000E3757C0A1220049000F6757C0BC9
:101DF000122004900109757C0C12200490011C75BE
:101E00007C0D12200490012F757C0E12200490018D
:101E100042757C0F122004229000AB757C051220C5
:101E2000049000BE757C071220049000D1757C09D7
:101E30001220049000E4757C0A1220049000F775CB
:101E40007C0B12200490010A757C0C122004900176
:101E50001D757C0D122004900130757C0E1220043B
:101E6000900143757C0F122004229000AC757C0514
:101E70001220049000BF757C071220049000D275D8
:101E80007C091220049000E5757C0A122004900061
:101E9000F8757C0B12200490010B757C0C12200449
:101EA00090011E757C0D122004900131757C0E127C
:101EB0002004900144757C0F122004229000AD751F
:101EC0007C051220049000C0757C0712200490004D
:101ED000D3757C091220049000E6757C0A12200458
:101EE0009000F9757C0B12200490010C757C0C128B
:101EF000200490011F757C0D122004900132757C26
:101F00000E122004900145757C0F122004229000CF
:101F1000AE757C051220049000C1757C0712200468
:101F20009000D4757C091220049000E7757C0A1299
:101F300020049000FA757C0B12200490010D757C32
:101F40000C122004900120757C0D122004900133A6
:101F5000757C0E122004900146757C0F122004221D
:101F60009000AF757C051220049000C2757C0712AA
:101F700020049000D5757C091220049000E8757C3F
:101F80000A1220049000FB757C0B12200490010EB5
:0E1F9000757C0C122004900121757C0D12202E
:101F9E0004900134757C0E122004900147757C0F5D
:101FAE00122004229000B0757C051220049000C30C
:101FBE00757C071220049000D6757C0912200490BF
:101FCE0000E9757C0A1220049000FC757C0B12202F
:101FDE000490010F757C0C122004900122757C0D6B
:101FEE00122004900135757C0E1220049001487564
:101FFE007C0F12200422E004B57C027400F02290C3
:10200E000194E0B40202D2B69001ABE0B40202D267
:10201E00B52230490BC2499004B8E0149004B7F0D1
:10202E002290018FE01214A3E090014BF090018FEB
:10203E00E0FF9006EB12140DE090014DF02290019E
:10204E008FE090007AE090014BF090018FE0FF90CE
:10205E0006EB12140DE090014DF02212202F0220FB
:10206E007212204C90014BE0B4000312207D22909E
:10207E00014DE07012F9900193E0B403099004B899
:10208E00E0149004B7F0E9041220E42274009001E9
:10209E004DF022740090014BF02274009004B7F0C2
:1020AE0022B408030220B75012F990018EE075F0A9
:1020BE0002A414149078D7930220DBC39408F990ED
:1020CE00018EE075F002A414149078D89323D9FDF4
:1020DE00A2E012210522B408030220EC5008F99068
:1020EE000198E00220FCC39408F9900199E023D9ED
:1020FE00FDA2E012210522400C900192E014700125
:10210E0022125C922212358A740090014CF0125CFD
:10211E00929006D7E02BF57390018DE060061221A8
:10212E00420221381222BD12215F900194E0B401C7
:10213E0002D2B6221222BDE573B5740302215F509E
:10214E0005C214022156D21412219EC21285737436
:10215E0022D212E573F5741205EBC2AD8582448569
:10216E008345D2AD2290014CE0F57C90019DE0B507
:10217E007C041221912240FA12218A2290014CE015
:10218E0004F0221222FF900194E0B40102C2B622A2
:10219E0020142CE5741205EBC2AD8582448583456F
:1021AE00D2ADE574C39573F5791205EB858259E5C9
:1021BE0082700375590185835A055A1221F922E559
:1021CE00741205EBC2AD858244858345D2ADE573AD
:1021DE00C39574F5791205EB858259E58270037506
:1021EE00590185835A055A1221F92290018DE0FA80
:1021FE007480C39AF5437537F175384E7539047589
:10220E003A00783785793B753C00793B1203998605
:10221E0037088638753900753A00783785433B752F
:10222E003C00793B1203998637088638753900755C
:10223E003A007837900189E02414F53B753C00791B
:10224E003B1203998682088683C2AD85825BE58246
:10225E007003755B0185835C055C855B5D855C5EEB
:10226E00D2AD22D55905D55A03D212227559FF2265
:10227E00301201222014030222A212227130120106
:10228E0022E5442401F582E5453400F58385824438
:10229E008583452212227130120122C3E544940136
:1022AE00F582E5459400F583858244858345229029
:1022BE0002B6E070041222FF22129F4DF5709001BB
:1022CE0095E0B4010FE57012061BC2AD85824C85F8
:1022DE00834DD2AD1222FF900201E02490120E180F
:1022EE00E5732424C2E7120E18E570120E18D234CC
:1022FE002220340122900201E02490120E18E5747F
:0E230E002424C2E7120E187400120E18C234F6
:10231C0022304A0BC24A90066DE01490066CF022F3
:10232C009001A6E01214A37400E090014EF090010D
:10233C00A6E0FF9006EC12140DE0900150F02290F4
:10234C0001A6E090007CE090014EF09001A6E0FF29
:10235C009006EC12143FE0900150F02212232C0254
:10236C00237112234B90014EE0B4000312237C2204
:10237C00900150E07012F99001AAE0B403099006A4
:10238C006DE01490066CF0E9041223E322740090C3
:10239C000150F022740090014EF022740090066CF3
:1023AC00F022B408030223B65012F99001A5E0758F
:1023BC00F002A414149078D7930223DAC39408F98A
:1023CC009001A5E075F002A414149078D89323D949
:1023DC00FDA2E012240422B408030223EB5008F9F6
:1023EC009001AFE00223FBC39408F99001B0E02305
:1023FC00D9FDA2E012240422400C9001A9E0147033
:10240C00012212645022123E1F740090014FF012F0
:10241C0064509006D7E02BF5769001A4E06006128C
:10242C0024410224371225BC12245E9001ABE0B487
:10243C000102D2B5221225BCE576B5770302215FE5
:10244C005005C215022455D21512249DC21385764F
:10245C007722D213E576F5771205EBC2AD8582466D
:10246C00858347D2AD2290014FE0F57C9001B4E01A
:10247C00B57C041224902240FA1224892290014F38
:10248C00E004F0221225FE9001ABE0B40102C2B5CB
:10249C002220152CE5771205EBC2AD85824685838B
:1024AC0047D2ADE577C39576F57A1205EB85825F59
:1024BC00E5827003755F0185836005601224F82244
:1024CC00E5771205EBC2AD858246858347D2ADE533
:1024DC0076C39577F57A1205EB85825FE5827003FA
:1024EC00755F0185836005601224F8229001A4E0D9
:1024FC00FA7480C39AF5437537F175384E75390403
:10250C00753A007837857A3B753C00793B12039914
:10251C008637088638753900753A00783785433B1D
:10252C00753C00793B12039986370886387539005B
:10253C00753A007837900189E02414F53B753C001E
:10254C00793B1203998682088683C2AD858261E548
:10255C0082700375610185836205628561638562A2
:10256C0064D2AD22D55F05D56003D21322755FFF0F
:10257C0022301301222015030225A11225703013DD
:10258C000122E5462401F582E5473400F583858276
:10259C00468583472212257030130122C3E54694E9
:1025AC0001F582E5479400F58385824685834722B1
:1025BC0090056BE070041225FE22129F98F5719025
:1025CC0001ACE0B4010FE57112061BC2AD85824E61
:1025DC0085834FD2AD1225FE900202E02490120E9C
:1025EC0018E5762424C2E7120E18E571120E18D2E3
:1025FC00352220350122900202E02490120E18E5BB
:10260C00772424C2E7120E187400120E18C2352259
:10261C007E011226457E021226457E031226457E39
:10262C00041226457E051226457E061226457E0797
:10263C001226457E08122645229001C012269DE0E6
:10264C001214A3E090015112269DF09001C01226A5
:10265C009DE0FF9006ED12269D12140DE090016195
:10266C0012269DF0229001C012269DE090007EE083
:10267C0090015112269DF09001C012269DE0FF9012
:0E268C0006ED12269D121471E09001611226D7
:10269A009DF022C0E08582378583387837EE14F5BD
:1026AA003B753C00793B12036E8682088683D0E034
:1026BA0022C0E08582378583387837EE1475F002B8
:1026CA00A4F53B753C00793B12036E86820886832B
:1026DA00D0E02290015112269DE0B400031226EBAD
:1026EA002290016112269DE004122746227400906E
:1026FA00016112269DF022740090015112269DF06C
:10270A0022B408030227135015FF9001B812269D20
:10271A00E075F002A414149078D79302273DC3946D
:10272A0008FF9001B812269DE075F002A4141490D7
:10273A0078D89323DFFDA2E012276D22B4080302A2
:10274A00274E500BFF9001E91226BBE0022764C313
:10275A009408FF9001EA1226BBE023DFFDA2E012F3
:10276A00276D224001221227861250611227867491
:10277A000090015912269DF01227B42290017DE0A3
:10278A00CEF02290015912269DE0F57C9001E112CB
:10279A00269DE0B57C041228012240FA1227AA22BB
:1027AA0090015912269DE004F022BE01074352010E
:1027BA001228D022BE02074352021228EB22BE037D
:1027CA000743522012290622BE0407435204122943
:1027DA002122BE050743524012293C22BE06074366
:1027EA00520812295722BE07074352801229722221
:1027FA0043521012298D22BE01075352FE1229A8F4
:10280A0022BE02075352FD1229C722BE03075352A2
:10281A00DF1229E622BE04075352FB122A0522BE02
:10282A0005075352BF122A2422BE06075352F71233
:10283A002A4322BE070753527F122A62225352EFBB
:10284A00122A81225352FE1229A85352FD1229C775
:10285A005352DF1229E65352FB122A055352BF1272
:10286A002A245352F7122A4353527F122A6253528E
:10287A00EF122A81227E011226717E021226717EB1
:10288A00031226717E041226717E051226717E06B7
:10289A001226717E071226717E081226717E011297
:1028AA0026DD7E021226DD7E031226DD7E04122636
:1028BA00DD7E051226DD7E061226DD7E071226DD66
:1028CA007E081226DD22900204E02490120E18746B
:1028DA0024120E187464120E189006F5E0D2E0F075
:1028EA0022900204E02490120E187425120E187415
:1028FA006E120E189006F5E0D2E1F022900204E082
:10290A002490120E18743C120E187478120E189035
:10291A0006F5E0D2E2F022900204E02490120E18AA
:10292A00743F120E18747F120E189006F5E0D2E367
:10293A00F022900204E02490120E187430120E183D
:10294A00746E120E189006F5E0D2E4F0229002049A
:10295A00E02490120E18743B120E18747F120E188F
:10296A009006F5E0D2E5F022900204E02490120EDF
:10297A0018743D120E18747F120E189006F5E0D2E4
:10298A00E6F022900204E02490120E18743E120E11
:10299A0018747F120E189006F5E0D2E7F02290061E
:1029AA00F5E020E00122C2E0F0900204E024901257
:1029BA000E187424120E187400120E18229006F5BE
:1029CA00E020E10122C2E1F0900204E02490120E1C
:1029DA00187425120E187400120E18229006F5E0CB
:1029EA0020E20122C2E2F0900204E02490120E18C2
:1029FA00743C120E187400120E18229006F5E0208C
:0E2A0A00E30122C2E3F0900204E02490120ED9
:102A180018743F120E187400120E18229006F5E072
:102A280020E40122C2E4F0900204E02490120E187F
:102A38007430120E187400120E18229006F5E02059
:102A4800E50122C2E5F0900204E02490120E187409
:102A58003B120E187400120E18229006F5E020E6BC
:102A68000122C2E6F0900204E02490120E18743D90
:102A7800120E187400120E18229006F5E020E701D5
:102A880022C2E7F0900204E02490120E18743E125D
:102A98000E187400120E1822122D5FE56B30E7072E
:102AA800122B88122D3422122B64122B76122AB97B
:102AB8002290017CE01475F006A4902AC673906DEC
:102AC800FB022B02906E01022B02906E07022B0272
:102AD800906E0D022B02906E13022B02906E19025B
:102AE8002B02906E1F022B27906E25022B02906EF0
:102AF8002B022B02906E31022B4C05A29000427BD8
:102B080006129176906DC805A29000487B0A129132
:102B180076906DC805A29000527B1012917622051E
:102B2800A29000427B05129176906DC805A2900094
:102B3800477B0B129176906DC805A29000527B10CE
:102B48001291762205A29000427B10129176906D28
:102B5800C805A29000527B10129176222002012211
:102B6800C20590017CE004120B0EF0C20222200381
:102B78000122C20590017CE014120B0EF0C2032260
:102B8800E56B20E50122E56B30E60122E56A30E0DD
:102B98002130E12730E22730E32730E52730E727E7
:102BA800E56B30E02530E10D30E20430E30A220223
:102BB8002BD5022BE4022BF3022C02022C11022C3F
:102BC80020022C2F022C38022C47022C509001880E
:102BD8007401F0740190017CF0022C5D90018874FE
:102BE80001F0740290017CF0022C5D90018874025F
:102BF800F0740390017CF0022C5D9001887403F05E
:102C0800740490017CF0022C5D9001887401F074CA
:102C18000590017CF0022C5D9001887401F0740627
:102C280090017CF0022C5D740790017CF0022C5D11
:102C38009001887401F0740890017CF0022C5D7496
:102C48000990017CF0022C5D740A90017CF0022C42
:102C58005D90017CE0B40106906DFB022CA6B402E5
:102C680006906E01022CA6B40303022CB4B404032C
:102C7800022CC8B40506906E13022CA6B406069062
:102C88006E19022CA6B40703022CDCB40806906E59
:102C980025022CF0B40906906E2B022CA622122DC8
:102CA8000405A29000427B0612917622906E0712CC
:102CB8002D0405A29000427B06129176122D112256
:102CC800906E0D122D0405A29000427B061291769B
:102CD800122D1122906E1F122D0405A29000427B26
:102CE80005129176124C8C22906E25122D0405A2A5
:102CF8009000427B0512917612520E222220080182
:102D08002220050122906DE822305206906FC902F8
:102D18002D29205306906FC1022D29906FC5022DD1
:102D28002905A29000477B041291762290017CE04D
:102D38001475F003A4902D4173022D9B0239DD0216
:102D48003F6502415F0243DF0247A8024CC10252BD
:102D5800430254A50258A4E56B30E703C2072220BA
:102D68000704B208D2072220020122C20590017E80
:102D7800E004120B21F090017FF0C202222003012F
:0E2D880022C20590017EE014120B21F0900192
:102D96007FF0C20322E56B20E50122C253128E2783
:102DA600122EDE122E89300807122D6F122D852263
:102DB60090017EE0B4010A122F5B122F6F128B94E2
:102DC60022B4020A1233C91233DD128B9422B403E1
:102DD6000A12346B12347F128B9422B4040A123412
:102DE600B81234CA128B9422B4051F123043123023
:102DF6005C12067A12095412091512093C900188D0
:102E06007404F09001797401F022B406159001FD66
:102E1600E0B40404128B94221232A11232B5128B42
:102E26009422B407159001FDE0B40404128B942299
:102E360012350E123520128B9422B4080A1235C8A8
:102E46001235DA128B9422B4090A12368A12369C8B
:102E5600128B9422B40A0A1236D21236E4128B94DA
:102E660022B40B159001FDE0B40404128B942212D7
:102E76003720123734128B942212377F1237911271
:102E86008B942290017EE0B40104122F8322B402B7
:102E9600041233F122B4030412349322B40404124C
:102EA60034DC22B405041230FE22B406041232E1E8
:102EB60022B4070412353222B408041235EC22B4C7
:102EC60009041236AE22B40A041236F622B40B04F2
:102ED600123748221237A32290017EE01475F006BD
:102EE600A4902EEB7390703F022F33907049022FFF
:102EF60033907053022F3390705D022F33907067BA
:102F0600022F41907071022F3390707B022F339005
:102F16007085022F3390708F022F33907099022F95
:102F2600339070A3022F339070AD022F33122F4FC0
:102F360005A29000487B0A12917622122F4F05A215
:102F46009000487B05129176222008012220050177
:102F560022906DE82220020122C20590018AE00437
:102F6600120BB9F0C202D2322220030122C205900E
:102F7600018AE014120BB9F0C203D2322290018A00
:102F8600E01475F006A4902F9073907265023038A5
:102F960090727502303890728502303890729502C0
:102FA60030389072A50230389072B502303890727F
:102FB600C50230389072D50230389072E50230384A
:102FC6009072F5023038907305023038907315020E
:102FD600303890732502303890733502303890734C
:102FE6004502303890735502303890736502303898
:102FF600907375023038907385023038907395025D
:1030060030389073A50230389073B502303890731B
:10301600C50230389073D50230389073E5023038E7
:103026009073F502303890740502303890741502AA
:10303600303805A29000527B1012917622200201B0
:1030460022C20590018EE0F904120C9AF0C2021217
:1030560032041231222220030122C20590018EE0A1
:10306600F914120C9AF0C20312320412312222E031
:10307600B4800302308E50FB1230A19000501291A2
:10308600AF90004F7450F022C3947F1230A190008D
:10309600501291AF90004F7455F022B42001224097
:1030A600FDB43F04C394202240FAC3944075F0084F
:1030B60084E5F00422E01475F005A49030C573741D
:1030C600100230F7740C0230F774050230F77407FB
:1030D6000230F774090230F7740A0230F7740B02F3
:1030E60030F7740D0230F7740E0230F7740F0230A9
:1030F600F790004D1291AF2290018E123075900616
:0E310600EB1230BB90018EE060041231962275
:10311400906E4105A29000527B101291762290018C
:103124008EE0B4800302313450FB1231590231373E
:103134001294F69001A5E0600122900199E0F490C8
:1031440001B0F0900198E0F49001AFF09006EBE04C
:103154009006ECF02290018EE070139001B0E0F440
:10316400900199F09001AFE0F4900198F022900161
:103174008E123182900199F0900198EFF022E0755F
:10318400F002A41414FB9078D793FFEB049078D743
:1031940093221232439001981231A912324A9001BB
:1031A400991231CB227408C39FFBE005A290005210
:1031B40023FAA2E01231FCF0A3EADFF4EB7001225F
:1031C4007420F0A3DBFA22EF700C7B0890005A7491
:1031D40020F0A3DBFA227408C39FFBE005A2900051
:1031E4005A23FAA2E01231FCF0A3EADFF4EB7001F7
:1031F400227420F0A3DBFA22400374A52274FF2278
:1032040090018EE070099006ECE09006EBF022B499
:103214008006C3947F02321E50F81232269006EBC9
:10322400F022B4200374012240FBB43F0374022251
:1032340040FBC3944075F008842403120A82229050
:1032440006EB123251229006EB12327922E0147509
:10325400F003A490325B737F08227F08227F05224B
:103264007F07227F08227F08227F08227F08227F8F
:1032740008227F0822E01475F003A4903283737F40
:1032840008227F04227F00227F00227F01227F0206
:10329400227F03227F05227F06227F07222002014C
:1032A40022C20590018FE004120CA6F0C202D2499A
:1032B4002220030122C20590018FE014120CA6F013
:1032C400C203D2492290018FE014B4100574600245
:1032D40032DC50F99077859390019CF0229001FDA7
:1032E400E0B404069077750233BE1232C990018FA0
:1032F400E01475F006A49032FE739076650233BE36
:103304009076750233BE9076850233BE9076950230
:1033140033BE9076A50233BE9076B50233BE907666
:10332400C50233BE9076D50233BE9076E50233BE35
:103334009076F50233BE9077050233BE907715027E
:1033440033BE9077250233BE9077350233BE907733
:10335400450233BE9077550233BE9077650233BE83
:103364009077750233BE9077850233BE90779502CD
:1033740033BE9077A50233BE9077B50233BE907703
:10338400C50233BE9077D50233BE9077E50233BED3
:103394009077F50233BE9078050233BE907815021B
:1033A40033BE9078250233BE9078350233BE9078D0
:1033B400450233BE9078550233BE05A29000527B7D
:1033C400101291762220020122C20590018BE004A2
:1033D400120BDFF0C202D2322220030122C2059076
:1033E400018BE014120BDFF0C203D2322290018B66
:1033F400E01460061475F003840475F006A4903498
:1034040006739073F502341E907405023429907487
:103414001502342990742502342905A29000527BA8
:10342400101291762205A29000527B0F1291769091
:10343400018BE0147001221234459000611291ABAB
:103444002290018BE01470037A0022B40403023446
:103454005F50037A0122B407005006C394037A0232
:1034640022C394067A032220020122C20590018C11
:10347400E004120CB9F0C202D2322220030122C2AB
:0E3484000590018CE014120CB9F0C203D23294
:1034920022906DC805A29000527B0712917690018E
:1034A2008CE09000591291AB90743D05A290005AA5
:1034B2007B081291762220020122C20590018DE042
:1034C20004120C05F0C2022220030122C20590015F
:1034D2008DE014120C05F0C2032290018DE0FA7403
:1034E2007FC39AB47F0302350090745505A2900001
:1034F200527B0D129176EA90005F1291C422907372
:10350200F505A29000527B10129176222002012230
:10351200C205900190E004120CCCF0C202222003FA
:103522000122C205900190E014120CCCF0C20322D9
:103532009001FDE0B404069077750233BE900190CD
:10354200E0B408041235642240FAB409069077A662
:1035520002357FB40A069077B602357F9077C602AD
:10356200357F90779605A29000527B0F129176904C
:103572000190E09000611291AB1235AF2205A2904A
:1035820000527B1012917622900190E0B40804025E
:1035920035AF2240FAB40906126CA20235B3B40A5E
:1035A20006126C980235B3126CAC0235B3900190DE
:1035B200E014F990018FE01475F008A429907816B0
:1035C2009390019DF02220020122C205900191E018
:1035D20004120C15F0C2022220030122C20590013E
:1035E20091E014120C15F0C20322900191E014B480
:1035F200100302366C50FB75F006A49036017390EE
:1036020075550236619075650236619075750236A0
:10361200619075850236619075950236619075A547
:103622000236619075B50236619075C502366190B9
:1036320075D50236619075E50236619075F50236F0
:103642006190760502366190761502366190762594
:103652000236619076350236619076450236610512
:10366200A29000527B1012917622C3940FFA7480BA
:10367200C39AFA90765505A29000527B0D1291766C
:10368200EA90005F1291C42220020122C205900139
:1036920092E004120C61F0C2022220030122C20550
:1036A200900192E014120C61F0C20322900192E0A8
:1036B2001475F006A49036BB739074650236C790F9
:1036C20074750236C705A29000527B1012917622C1
:1036D20020020122C205900193E004120C74F0C290
:1036E200022220030122C205900193E014120C74FD
:1036F200F0C20322900193E01475F006A490370300
:10370200739073F50237159074850237159074958E
:1037120002371505A29000527B10129176222002E8
:103722000122C205900194E004120C3BF0C202C2D5
:10373200B62220030122C205900194E014120C3B30
:10374200F0C203C2B6229001FDE0B404069074E513
:10375200023774900194E01475F006A490376273F6
:103762009074E50237749074F5023774907505020F
:10377200377405A29000527B10129176222002012A
:1037820022C205900195E004120C4EF0C2022220E2
:10379200030122C205900195E014120C4EF0C203FF
:1037A20022900195E01475F006A49037B0739075DD
:1037B200150237B990752505A29000527B1012911F
:1037C200762290017CE0B4090122B40A0122E56B61
:1037D20030E524203C0122D232C23C90017CE0B48C
:1037E20008329006BE1251EDE56C04F09006CA1242
:1037F20051EDE56F04F022D23C1238BB123931127E
:0E380200381A90021DE07003856C6D9004D2A0
:10381000E07003856F6E22302F229078A605A2906B
:1038200000527B0912917612384090017CE0B4037B
:1038300004123F5722B40403123F57221238B12218
:10384000E56C12387905A290005B7B0212917690AC
:103850006DC805A290005D7B01129176E56F12386C
:103860007905A290005E7B02129176906DC805A248
:103870009000607B021291762275F004A49038814A
:10388000739078AF229078B1229078B3229078B577
:10389000229078B7229078B9229078BB229078BD98
:1038A000229078BF229078C1229078C3229078C568
:1038B000225350FF4350DE4351D722E56B20E105F0
:1038C000740002392820E205740102392820E3053A
:1038D000740202392820E4057406023928E56A20BA
:1038E000E005740302392820E10574040239282018
:1038F000E205740502392820E305740702392820FF
:10390000E405740802392820E505740902392820E5
:10391000E605740A02392820E705740B02392820CD
:103920005303E56C22E56F22205303F56C22F56FFB
:103930002275F00AA4903939735350FD4350DC438B
:1039400051D7225350FB4350DA4351D7225350F7FB
:103950004350D64351D7225350EF4350CE4351D713
:10396000225350BF43509E4351D72253507F435060
:103970005E4351D7225351FE4351D64350DE22536A
:1039800051FD4351D54350DE225351FB4351D343A4
:1039900050DE225351EF4351C74350DE225351BFF3
:1039A0004351974350DE2253517F4351574350DEDA
:1039B0002220020122C20590017FE004120B21F0B7
:1039C00090017EF0C2022220030122C20590017FF5
:1039D000E014120B21F090017EF0C20322E56B206F
:1039E000E50122D253128E27123B20123ACB300827
:1039F000071239B11239C72290017FE0B4010A12CF
:103A00003B27123B3C128B9422B4020A123CA812B0
:103A10003CBC128B9422B4030A123D2B123D3F1280
:103A20008B9422B4040A123D78123D8A128B9422A0
:103A3000B4051F123B58123B7112068C12096B120F
:103A4000091512093C9001887405F0900179740100
:103A5000F022B406159001FDE0B40404128B942208
:103A6000123C51123C65128B9422B407159001FD53
:103A7000E0B40404128B9422123DA3123DB5128BC4
:103A80009422B4080A123E5D123E6F128B9422B447
:103A9000090A123E88123E9A128B9422B40A0A1224
:103AA0003EB3123EC5128B9422B40B159001FDE07B
:103AB000B40404128B9422123EDE123EF0128B9458
:103AC00022123F16123F2A128B942290017FE0B4FB
:103AD0000104123B5122B40204123CD022B403046C
:103AE000123D5322B40404123D9C22B40504123B3F
:103AF0008A22B40604123C9122B40704123DC72264
:103B0000B40804123E8122B40904123EAC22B40A65
:103B100004123ED722B40B04123F0222123F3E226F
:103B200090017FE0022EE220020122C2059001A155
:103B3000E004120BB9F0C20212A5242220030122D4
:103B4000C2059001A1E014120BB9F0C20312A52422
:103B5000229001A1E0022F8720020122C2059001DC
:103B6000A5E0F904120C9AF0C202123C21123BAEFD
:103B70002220030122C2059001A5E0F914120C9A3B
:0E3B8000F0C203123C21123BAE229001A512AE
:103B8E0030759006EC1230BB9001A5E06004123C3B
:103B9E000E22906E5105A29000527B101291762249
:103BAE009001A5E0B48003023BC050FB123BE5023E
:103BBE003BC312950990018EE06001229001B0E0A6
:103BCE00F4900199F09001AFE0F4900198F0900616
:103BDE00ECE09006EBF0229001A5E07013900199B5
:103BEE00E0F49001B0F0900198E0F49001AFF02273
:103BFE009001A51231829001B0F09001AFEFF0224A
:103C0E00123C439001AF1231A9123C4A9001B012FE
:103C1E0031CB229001A5E070099006EBE09006EC06
:103C2E00F022B48006C3947F023C3B50F812322639
:103C3E009006ECF0229006EC123251229006EC1215
:103C4E0032792220020122C2059001A6E004120C54
:103C5E00A6F0C202D24A2220030122C2059001A67A
:103C6E00E014120CA6F0C203D24A229001A6E01470
:103C7E00B410057460023C8C50F9907785939001D6
:103C8E00B3F0229001FDE0B404069077750233BEC6
:103C9E00123C799001A6E00232F520020122C20503
:103CAE009001A2E004120BDFF0C202D232222003F6
:103CBE000122C2059001A2E014120BDFF0C203D262
:103CCE0032229001A2E01460061475F0038404758C
:103CDE00F006A4903CE5739073F5023CFD907405DC
:103CEE00023D08907415023D08907425023D0805AA
:103CFE00A29000527B101291762205A29000527B68
:103D0E000F1291769001A2E014700122123D2490C0
:103D1E0000611291AB229001A2E00234492002010F
:103D2E0022C2059001A3E004120CB9F0C202D232F5
:103D3E002220030122C2059001A3E014120CB9F057
:103D4E00C203D23222906DC805A29000527B071298
:103D5E0091769001A3E09000591291AB90743D05BD
:103D6E00A290005A7B081291762220020122C205EF
:103D7E009001A4E004120C05F0C2022220030122DD
:103D8E00C2059001A4E014120C05F0C203229001AA
:103D9E00A4E00234E020020122C2059001A7E00453
:103DAE00120CCCF0C2022220030122C2059001A700
:103DBE00E014120CCCF0C203229001FDE0B4040614
:103DCE009077750233BE9001A7E0B40804123DF956
:103DDE002240FAB409069077A6023E14B40A069061
:103DEE0077B6023E149077C6023E1490779605A2DF
:103DFE009000527B0F1291769001A7E09000611215
:103E0E0091AB123E442205A29000527B1012917685
:103E1E00229001A7E0B40804023E442240FAB409FD
:103E2E0006126CA2023E48B40A06126C98023E4874
:103E3E00126CAC023E489001A7E014F99001A6E086
:103E4E001475F008A429907816939001B4F02220EE
:103E5E00020122C2059001A8E004120C15F0C20264
:103E6E002220030122C2059001A8E014120C15F0C5
:103E7E00C203229001A8E00235F020020122C20501
:103E8E009001A9E004120C61F0C20222200301226B
:103E9E00C2059001A9E014120C61F0C20322900138
:103EAE00A9E00236B220020122C2059001AAE00466
:103EBE00120C74F0C2022220030122C2059001AA44
:103ECE00E014120C74F0C203229001AAE00236FA3A
:103EDE0020020122C2059001ABE004120C3BF0C29D
:103EEE00022220030122C2059001ABE014120C3B0A
:0E3EFE00F0C203229001FDE0B404069074E5CA
:103F0C000237749001ABE002375920020122C2053E
:103F1C009001ACE004120C4EF0C202C2B522200398
:103F2C000122C2059001ACE014120C4EF0C203C287
:103F3C00B5229001ACE01475F006A4903F4B739041
:103F4C0075350237B99075450237B9906DC805A221
:103F5C0090004B7B0412917622E56B20E501221236
:103F6C003F78123FAE123FE4122D112220020122A3
:103F7C00C205305210900196E004120CF2F0900140
:103F8C00ADF0023FA920530C900196E004120CF204
:103F9C00F0023FA99001ADE004120CF2F0C202D283
:103FAC00362220030122C205305210900196E014F3
:103FBC00120CF2F09001ADF0023FDF20530C900197
:103FCC0096E014120CF2F0023FDF9001ADE01412F7
:103FDC000CF2F0C203D236222053139001961240F9
:103FEC0022123F5790019612414512944D22900196
:103FFC00AD124022123F579001AD12414512946010
:10400C0022900196124022123F5790019612414580
:10401C0012944D023FFAE0B42B06907D8802413495
:10402C0050F81475F006A490403773907AE802416A
:10403C0030907AF8024130907B08024130907B1826
:10404C00024130907B28024130907B380241309005
:10405C007B48024130907B58024130907B68024192
:10406C0030907B78024130907B88024130907B9875
:10407C00024130907BA8024130907BB802413090D5
:10408C007BC8024130907BD8024130907BE80241E2
:10409C0030907BF8024130907C08024130907C18C3
:1040AC00024130907C28024130907C3802413090A3
:1040BC007C48024130907C58024130907C6802412F
:1040CC0030907C78024130907C88024130907C9812
:1040DC00024130907CA8024130907CB80241309073
:1040EC007CC8024130907CD8024130907CE802417F
:1040FC0030907CF8024130907D08024130907D1860
:10410C00024130907D28024130907D380241309040
:10411C007D48024130907D58024130907D680241CB
:10412C0030907D781243902205A29000527B1012A1
:10413C00917690004F7455F022E0B42B0302415558
:10414C0050FB9000501291AF22C3942A9000501251
:10415C0091AF22E56B20E501221241721241A812A7
:10416C0041DE122D112220020122C2053052109084
:10417C000197E004120D05F09001AEF00241A3206E
:10418C00530C900197E004120D05F00241A390012D
:10419C00AEE004120D05F0C202D237222003012238
:1041AC00C205305210900197E014120D05F09001E9
:1041BC00AEF00241D920530C900197E014120D057A
:1041CC00F00241D99001AEE014120D05F0C203D2F9
:1041DC00372220531390019712421C123F57900123
:1041EC00971243A1129473229001AE12421C123FFB
:1041FC00579001AE1243A11294862290019712425D
:10420C001C123F579001971243A11294730241F470
:10421C00E0B437079083B51241342250F7B42B0326
:10422C00024231400BC3942B75F006A490434173AA
:10423C001475F006A49042457390805502438C90FF
:10424C00806502438C90807502438C90808502437C
:10425C008C90809502438C9080A502438C9080B505
:10426C0002438C9080C502438C9080D502438C9085
:0E427C0080E502438C9080F502438C90810512
:10428A0002438C90811502438C90812502438C90C5
:10429A00813502438C90814502438C9081550243BB
:1042AA008C90816502438C90817502438C90818544
:1042BA0002438C90819502438C9081A502438C9095
:1042CA0081B502438C9081C502438C9081D502430B
:1042DA008C9081E502438C9081F502438C90820593
:1042EA0002438C90821502438C90822502438C9063
:1042FA00823502438C90824502438C908255024358
:10430A008C90826502438C90827502438C908285E0
:10431A0002438C90829502438C9082A502438C9032
:10432A0082B502438C9082C502438C9082D50243A7
:10433A008C9082E502438C9082F502438C9083052F
:10434A0002438C90831502438C90832502438C9000
:10435A00833502438C90834502438C9083550243F4
:10436A008C90836502438C90837502438C9083857D
:10437A0002438C90839502438C9083A502438C90D0
:10438A0083B51243902205A29000527B10129176B7
:10439A0090004F7450F022E0B437030243B150FB4F
:1043AA009000501291AF22C394369000501291AFF0
:1043BA002220020122C205900182E004120B47F07A
:1043CA00C2022220030122C205900182E014120BCC
:1043DA0047F0C20322E56B20E50122128B94128E6C
:1043EA00271244991244593008071243BB1243CD8D
:1043FA0022900182E0B4010A304F061244EA1244C4
:10440A00FC22B4020712454A12455F22B40307127E
:10441A0045B11245C322B404071245F912460B22CC
:10442A00B4050712465112466322B4060712469093
:10443A001246A222B407071246CD1246DF22B4085A
:10444A000712470A12471C2212474712475922905D
:10445A000182E0B4010412450E22B402041245811D
:10446A0022B403041245D522B4040412461D22B410
:10447A00050412467522B406041246B422B407048F
:10448A001246F122B4080412472E2212476B2290D8
:10449A000182E01475F006A49044A6739070D702C6
:1044AA0044DC9070E10244DC9070EB0244DC9070D2
:1044BA00F50244DC9070FF0244DC9071090244DC8E
:1044CA009071130244DC90711D0244DC9071270242
:1044DA0044DC122F4F05A29000487B0A12917622E3
:1044EA0020020122C205900189E004120A2CF0C2BE
:1044FA00022220030122C205900189E014120A2C2B
:10450A00F0C203229001FDE0B4021A906DC805A220
:10451A009000527B0D129176900189E0241490004C
:10452A005F1291C422906DC805A29000527B0A12B4
:10453A00917690713105A290005C7B0612917622E9
:10454A0020020122C2059001FDE004120C28F0C2EB
:10455A00021245742220030122C2059001FDE014D3
:10456A00120C28F0C203124574229001FDE0147067
:10457A0003C24F22D24F229001FDE01475F006A427
:10458A0090458E739071310245A69071410245A6FD
:10459A009071510245A69071610245A605A290004C
:1045AA00527B101291762220020122C205D2599022
:1045BA0001FEE0D2E2F0C2022220030122C205C2B9
:1045CA00599001FEE0C2E2F0C20322906DC805A232
:1045DA009000527B0A129176205906907171024519
:1045EA00EE90717705A290005C7B061291762220EC
:0E45FA00020122C2059001FCE004120B5AF0EF
:10460800C2022220030122C2059001FCE014120B11
:104618005AF0C20322906DC805A29000527B0A127C
:1046280091769001FCE01475F006A49046377390DB
:10463800717D02464690717102464690717705A2D7
:1046480090005C7B061291762220020122C205901E
:104658000200E004120A3CF0C2022220030122C236
:1046680005900200E014120A3CF0C20322906DC8C3
:1046780005A29000527B0E129176900200E0F56937
:10468800049000601291AF2220020122C20590021C
:1046980001E004120A3CF0C2022220030122C205F2
:1046A800900201E014120A3CF0C20322906DC80582
:1046B800A29000527B0E129176900201E0049000C5
:1046C800601291AF2220020122C205900202E0048A
:1046D800120A3CF0C2022220030122C20590020203
:1046E800E014120A3CF0C20322906DC805A29000A3
:1046F800527B0E129176900202E0049000601291B3
:10470800AF2220020122C205900203E004120A3CF3
:10471800F0C2022220030122C205900203E0141213
:104728000A3CF0C20322906DC805A29000527B0E8D
:10473800129176900203E0049000601291AF22205B
:10474800020122C205900204E004120A3CF0C202EF
:104758002220030122C205900204E014120A3CF050
:10476800C20322906DC805A29000527B0E1291766A
:10477800900204E0049000601291AF22200201220E
:10478800C205900183E004120B93F0C202222003B9
:104798000122C205900183E014120B93F0C2032298
:1047A800E56B20E50122128B94128E271247F9122D
:1047B80047E330080712478412479622900183E0A6
:1047C800B4010712485312486522B402071249E699
:1047D8001249F822124B79124B8B22900183E0B4D4
:1047E800010412487722B40204124A0A22124B9D8D
:1047F80022900183E01475F006A490480673907126
:104808008302481890718D024818907197024818D1
:10481800122F4F05A29000487B0A12917622300889
:104828002205A2900183E0B4010B9001F9E0900603
:10483800E8F0024848B402089001FAE09006E9F06E
:1048480005A22220050122906DE82220020122C241
:10485800059001F9E004120BCCF0C20222200301FA
:1048680022C2059001F9E014120BCCF0C203229089
:1048780001F9E01475F006A4904884739071E3027E
:1048880049509071EE0249509071F9024950907266
:104898000402495090720F02495090721A0249500E
:1048A80090722502495090723002495090723B0232
:1048B80049509072460249509071F902496E9072BF
:1048C8000402496E90720F02496E90721A02496E84
:1048D80090722502496E90723002496E9071F90209
:1048E800498C90720402498C90720F02498C907224
:1048F8001A02498C90722502498C90723002498CB8
:104908009071F90249AA9072040249AA90720F02A2
:1049180049AA90721A0249AA9072250249AA90726D
:10492800300249AA9071F90249C89072040249C834
:1049380090720F0249C890721A0249C890722502F3
:1049480049C89072300249C812482605A2900057FB
:104958007B0B1291769071B112482605A2900052F5
:104968007B051291762212482605A29000577B0BF0
:0E4978001291769071B612482605A290005258
:104986007B051291762212482605A29000577B0BD2
:104996001291769071BB12482605A29000527B05B3
:1049A6001291762212482605A29000577B0B12918F
:1049B600769071C012482605A29000527B0512918E
:1049C600762212482605A29000577B0B129176900C
:1049D60071C512482605A29000527B0512917622D7
:1049E60020020122C2059001FAE004120BCCF0C2AB
:1049F600022220030122C2059001FAE014120BCC18
:104A0600F0C203229001FAE01475F006A4904A174A
:104A1600739071E3024AE39071EE024AE39071F9F2
:104A2600024AE3907204024AE390720F024AE3904C
:104A3600721A024AE3907225024AE3907230024AE1
:104A4600E390723B024AE3907246024AE39071F9A0
:104A5600024B01907204024B0190720F024B0190BF
:104A6600721A024B01907225024B01907230024B72
:104A7600019071F9024B1F907204024B1F90720F46
:104A8600024B1F90721A024B1F907225024B1F9009
:104A96007230024B1F9071F9024B3D907204024B2B
:104AA6003D90720F024B3D90721A024B3D9072255B
:104AB600024B3D907230024B3D9071F9024B5B9078
:104AC6007204024B5B90720F024B5B90721A024BA0
:104AD6005B907225024B5B907230024B5B1248264C
:104AE60005A29000577B0B1291769071CA12482648
:104AF60005A29000527B051291762212482605A245
:104B06009000577B0B1291769071CF12482605A222
:104B16009000527B051291762212482605A290003B
:104B2600577B0B1291769071D412482605A29000FD
:104B3600527B051291762212482605A29000577BD9
:104B46000B1291769071D912482605A29000527BDD
:104B5600051291762212482605A29000577B0B1269
:104B660091769071DE12482605A29000527B0512BE
:104B760091762220020122C205900187E004120BE1
:104B8600A6F0C2022220030122C205900187E0148A
:104B9600120BA6F0C203229071A105A29000527BCF
:104BA6000E129176900187E0149000601291AB90FE
:104BB60071B005A29000617B01129176124BC6225C
:104BC600300E0122900187E01475F00CA41205EB5B
:104BD600C2AD858244858345858246858347D2ADAD
:104BE600900187E01475F00CA4120603C2AD85820D
:104BF6004885834985824A85834B85824C85834DCA
:104C060085824E85834FD2AD2290017DE0F9124C0C
:104C16001AE9F022E56B44E1F47006E56AF47015D2
:104C26002230E10379012230E2012230E3037902E6
:104C36002230E40122E56AF430E0012230E1037912
:104C4600032230E20379042230E30379052230E4BB
:104C5600012230E50379062230E60379082230E79F
:104C66000379072222C0E08582378583387837901A
:104C7600017DE014F53B753C00793B12036E86829C
:104C8600088683D0E02290017DE09000471291AB28
:104C96009000487420F02220020122C2059001846F
:104CA600E004120B34F0C2022220030122C2059056
:104CB6000184E014120B34F0C20322E56B20E601F6
:104CC6002220E50122124C0F124C8C124D26124D59
:104CD60010300807124C9D124CAF22900184E0B4AC
:104CE6000107124D61124D7D22B4020F9001FDE0C5
:0E4CF600B4040122124F35124F4D229001FDE1
:104D0400E0B4040122124FD8124FED22900184E046
:104D1400B40104124DC722B40204124F652212508A
:104D24000222900184E01475F006A4904D33739030
:104D34007067024D53907072024D4590707C024D25
:104D440045122F4F05A29000497B09129176221239
:104D54002F4F05A29000487B051291762220020174
:104D640022C2059001B8124C6BE0F904120C9AF0BF
:104D7400C202124D99124DFD2220030122C2059058
:104D840001B8124C6BE0F914120C9AF0C203124DE4
:104D940099124DFD229001B8124C6BE0700F9006F1
:104DA400ED124E8DE09006ED124C6BF022B48006AD
:104DB400C3947F024DBC50F81232269006ED124C7B
:104DC4006BF0229001B8124C6B1230759006ED1204
:104DD4004C6B1230BB9001B8124C6BE06004124F64
:104DE4000822906E6105A29000527B0F12917612F8
:104DF4004ED19000611291AB229001B8124C6BE03D
:104E0400B48003024E1250FB124E4C024E15129502
:104E14001C9001B8124E8DE06001229001EA124EFE
:104E2400E3E0F49001EA124EADF09001E9124EE392
:104E3400E0F49001E9124EADF09006ED124C6BE0F7
:104E44009006ED124E8DF0229001B8124C6BE0707A
:104E54001F9001EA124EADE0F49001EA124EE3F025
:104E64009001E9124EADE0F49001E9124EE3F02214
:104E74009001B8124C6B1231829001EA124EE3F0A9
:104E84009001E9124EE3EFF022C0E085823785837A
:104E9400387837124ED114F53B753C00793B120338
:104EA4006E8682088683D0E022C0E08582378583BF
:104EB400387837124ED11475F002A4F53B753C00D6
:104EC400793B12036E8682088683D0E02290017DAE
:104ED400E0B40506C39404024EE250F8240422C050
:104EE400E0858237858338783790017DE01475F04A
:104EF40002A4F53B753C00793B12036E868208865A
:104F040083D0E022124F219001E9124EE31231A91D
:104F1400124F2B9001EA124EE31231CB229006ED90
:104F2400124C6B123251229006ED124C6B123279F4
:104F34002220020122C2059001C0124C6BE004122F
:104F44000CA6F0C202124F9F2220030122C2059038
:104F540001C0124C6BE014120CA6F0C203124F9F56
:104F6400229001FDE0B404079077751233BE22123B
:104F74004F819001C0124C6BE01232F5229001C0B7
:104F8400124C6BE014B410057460024F9750F99002
:104F94007785939001D0124C6BF02290017DE01440
:104FA40075F005A4904FAC737901024FD1790202D8
:104FB4004FD17904024FD17908024FD17910024FB1
:104FC400D17920024FD17940024FD179809001D814
:104FD400E049F02220020122C2059001D9124C6B53
:104FE400E004120CCCF0C2022220030122C205907C
:104FF40001D9124C6BE014120CCCF0C203229001C4
:10500400FDE0B404079077751233BE229001D912E3
:105014004C6BE0B408041250382240FAB4090690EC
:1050240077A6025056B40A069077B6025056907787
:10503400C602505690779605A29000527B0F1291AB
:10504400769001D9124C6BE09000611291AB125032
:10505400892205A29000527B10129176229001D9E8
:10506400124C6BE0B408040250892240FAB40906D9
:0E507400126CA2025090B40A06126C98025000
:1050820090126CAC0250909001D9124C6BE014FF5C
:105092009001C0124C6BE01475F008A42F907816A2
:1050A200939001E1124C6BF02220570122C2571259
:1050B20050FF4350DE4351D7E550C2E0F550D23A9B
:1050C200D23AD23B125114128B64125D1112513337
:1050D200128B7C1264CF1250DC22900186E0B40164
:1050E2000990022A128CB2028BA6B402099004DF44
:1050F200128CDB028BA64350DE4351D7229006BEB0
:105102001251EDE014F56C9006CA1251EDE014F55F
:105112006F229006A61251EDE0B43A08900196F083
:105122001297762240F6C3943A900197F0129BBEF2
:10513200229006B21251EDE0B43A089001ADF0129D
:10514200982B2240F6C3943A9001AEF0129BD622DD
:10515200E56B20E50122900186E0B4030122900173
:1051620085E0F912516BE9F022E56B44E1F4700835
:10517200E56AF47028C2582220586FD25830E105EF
:1051820079010251E930E20579020251E930E30581
:1051920079030251E930E40579070251E920584ABE
:1051A200D258E56AF430E00579040251E930E105AC
:1051B20079050251E930E20579060251E930E30549
:1051C20079080251E930E40579090251E930E5052F
:1051D200790A0251E930E605790B0251E930E70517
:1051E200790C0251E9790CD2572222C0E08582372C
:1051F2008583387837900185E014F53B753C00795A
:105202003B12036E8682088683D0E022900185E0FD
:105212009000471291AF2220020122C2059001861E
:10522200E004120B80F0C2021250DC2220030122A1
:10523200C205900186E014120B80F0C2031250DC0A
:1052420022E56B20E50122E56B20E6012212515294
:105252001252B012528E30080712521912522E22D6
:10526200900186E0B4010C1252EB125302C25312A7
:1052720050DC22B4020C12538612539DD2531250A8
:10528200DC221253F11254031250DC22900186E008
:10529200B4010A12520E12542D12531922B4020AE8
:1052A20012520E1254571253B42212541522900164
:1052B20086E01475F006A49052BD73906E7202528D
:1052C200CF906E750252CF906E810252DD122F4F37
:1052D20005A29000497B0112917622122F4F05A25E
:1052E2009000467B0C1291762220020122C2059088
:1052F20006A61251EDE004120D18F0D257C2022296
:1053020020030122C2059006A61251EDE014120DEF
:1053120018F0D257C2032212531D229006A6125130
:10532200EDE0B43A131240239006A61251ED124159
:1053320045906E791253562240EBC3943A12421DA5
:105342009006A61251EDE0C3943A1243A2906E7BEE
:105352001253562205A290004E7B011291762290A2
:105362006E7705A29000487B021291769006D7E0F4
:1053720090004A1291AF906DC805A290004C7B013B
:105382001291762220020122C2059006B21251ED3C
:10539200E004120D18F0D257C2022220030122C2E9
:1053A200059006B21251EDE014120D18F0D257C258
:1053B20003221253B8229006B21251EDE0B43A130E
:1053C2001240239006B21251ED124145906E7912AD
:1053D20053562240EBC3943A12421D9006B2125128
:1053E200EDE0C3943A1243A2906E7B1253562220F0
:0E53F200020122C2059006D6E004120D64F0FE
:10540000C2022220030122C2059006D6E014120D2A
:1054100064F0C20322906DC805A29000527B0E1268
:1054200091769006D6E09000601291AF22906DC800
:1054300005A290004A7B01129176E56C123879053D
:10544000A290004B7B02129176906DC805A290004D
:105450004D7B0112917622906DC805A290004A7B87
:1054600001129176E56F12387905A290004B7B020C
:10547000129176906DC805A290004D7B0112917635
:105480002220020122C205900188E004120B6DF077
:10549000C2022220030122C205900188E014120BEF
:1054A0006DF0C20322303C0122128B94128E27121F
:1054B00055301254FF125706300807125481125407
:1054C0009322900188E01475F003A49054CF7302E6
:1054D00054DE0254E30254EA0254F10254F8C202C8
:1054E000C203221255C51255D7221255F412560680
:1054F0002212562312562F221256D51256E122900E
:105500000176E060012290701F05A29000527B108E
:105510001291762290702F05A29000527B1012916A
:105520007622906DB805A29000527B1012917622DF
:10553000900188E01475F006A490553D73906FEDCE
:1055400002555B906FF702556990700102557A9091
:10555000700B02558B9070150255A8122F4F05A2A3
:105560009000487B0A12917622122F4F05A29000DC
:10557000487B081291761255E922122F4F05A2900E
:1055800000487B0812917612561822122F4F05A25E
:105590009000487B051291769006EB1230BB745553
:1055A00090004FF01256FB22122F4F05A290004898
:1055B0007B051291769006EC1230BB745590004F2B
:1055C000F01256FB2220020122C205900177E0046E
:1055D000120A6FF0C2022220030122C20590017755
:1055E000E014120A6FF0C20322900177E09000509D
:1055F0001291AF2220020122C205900178E004122C
:105600000A6FF0C2022220030122C205900178E055
:1056100014120A6FF0C20322900178E09000501239
:1056200091AF2220020122C20512563BC202222063
:10563000030122C205125642C203229006EB125603
:1056400049229006EB12568F22E01475F003A490C5
:1056500056537302567102567B02568502568502D6
:105660005685025685025685025685025685025693
:1056700085900179E004120A95F022900179E00406
:10568000120AA8F022900179E004120ABBF022E08D
:105690001475F003A4905699730256B70256C102CE
:1056A00056CB0256CB0256CB0256CB0256CB0256F5
:1056B000CB0256CB0256CB900179E014120A95F03A
:1056C00022900179E014120AA8F022900179E014E6
:1056D000120ABBF02220020122C2051256EDC202BC
:1056E0002220030122C2051256F4C203229006ECC6
:1056F000125649229006EC12568F22900179E090C2
:1057000000501291AF22E56B30E5089001FEE0C237
:10571000E0F0229001FEE020E043D2E0F0125522BA
:1057200012035D900188E0B4010912956512955548
:10573000025754B4020612575E025754B4030612BD
:105740005769025754B4040612587C025754125831
:10575000900257541255149001767404F02220538D
:1057600004125774221257B6222053041257F822FB
:0E57700012583A2290066F05A290021DE01218
:10577E000A5FFA90020505A2F0A370057C0102579C
:10578E00A505A2E0C3940CC3956CA305A2F0A3DA01
:10579E00F090021DE004FC90017712960D05A2EC2C
:1057AE00FB90066F1294192290067C05A29004D2EB
:1057BE00E0120A5FFA9004BA05A2F0A370057C010C
:1057CE000257E705A2E0C3940CC3956FA305A2F0A0
:1057DE00A3DAF09004D2E004FC90017712960D0546
:1057EE00A2ECFB90067C1294192290068905A290D9
:1057FE00021DE0120A5FFA90020505A2F0A37005E1
:10580E007C0102582905A2E0C3940CC3956CA30534
:10581E00A2F0A3DAF090021DE004FC90017812963B
:10582E007E05A2ECFB90068912941922900696052D
:10583E00A29004D2E0120A5FFA9004BA05A2F0A375
:10584E0070057C0102586B05A2E0C3940CC3956FE2
:10585E00A305A2F0A3DAF09004D2E004FC90017844
:10586E0012967E05A2ECFB900696129419229006D3
:10587E00EB1296CC1296FE05A27B02900198129422
:10588E0019229006EC1296CC1296FE05A27B02907F
:10589E0001AF129419221258B1E56B20E6012212C3
:1058AE00515222906E8D05A29000427B011291768C
:1058BE00900185E09000431291AF906DC805A290C3
:1058CE0000457B01129176E56C12387905A29000A5
:1058DE00467B02129176906DC805A29000487B011E
:1058EE00129176125958906DC805A290004D7B0109
:1058FE00129176125A92906E9D05A29000527B01E3
:10590E001291769006D7E09000531291AF906DC829
:10591E0005A29000557B01129176E56F123879053C
:10592E00A29000567B02129176906DC805A290004F
:10593E00587B01129176125991906DC805A2900074
:10594E005D7B01129176125AB1229006A61251ED8C
:10595E00E0B43A131259E09006A61251ED125A2CE9
:10596E00906E791259CA2240EBC3943A1259F390B1
:10597E0006A61251EDE0C3943A125A46906E7B126F
:10598E0059CA229006B21251EDE0B43A13125A06D9
:10599E009006B21251ED125A5F906E791259D522BD
:1059AE0040EBC3943A125A199006B21251EDE0C36D
:1059BE00943A125A79906E7B1259D52205A2900014
:1059CE00497B011291762205A29000597B0112911A
:1059DE007622B42B0790004A7455F02250F79000AF
:1059EE004A7450F022B4350790004A7455F0225094
:1059FE00F790004A7450F022B42B0790005A745559
:105A0E00F02250F790005A7450F022B435079000EF
:105A1E005A7455F02250F790005A7450F022E0B4A8
:105A2E002B03025A3C50FB90004B1291AF22C394B1
:105A3E002A90004B1291AF22B43503025A5550FBF7
:105A4E0090004B1291AF22C3943490004B1291AF41
:105A5E0022E0B42B03025A6F50FB90005B1291AF01
:105A6E0022C3942A90005B1291AF22B43503025ADE
:105A7E008850FB90005B1291AF22C3943490005B70
:105A8E001291AF22300504125AD022906DC805A291
:105A9E0090004E7B011291769006E6E090004F1238
:105AAE0091C422300504125BB122906DC805A290FC
:105ABE00005E7B011291769006E7E090005F1291F6
:105ACE00C4229006E8E01475F006A4905ADD739097
:105ADE006EAD025BA6906EB1025BA6906EB5025BD8
:0E5AEE00A6906EB9025BA6906EBD025BA690FC
:105AFC006EC1025BA6906EC5025BA6906EC9025B7E
:105B0C00A6906ECD025BA6906ED1025BA6906ED570
:105B1C00025BA6906ED9025BA6906EDD025BA6902E
:105B2C006EE1025BA6906EE5025BA6906EE9025BED
:105B3C00A6906EED025BA6906EF1025BA6906EF5E0
:105B4C00025BA6906EF9025BA6906EFD025BA690BE
:105B5C006F01025BA6906F05025BA6906F09025B5A
:105B6C00A6906F0D025BA6906F11025BA6906F154D
:105B7C00025BA6906F19025BA6906F1D025BA6904C
:105B8C006F21025BA6906F25025BA6906F29025BCA
:105B9C00A6906F2D025BA6906F3105A290004E7BF4
:105BAC0004129176229006E9E01475F006A4905B3D
:105BBC00BE73906F39025C87906F3D025C87906F6B
:105BCC0041025C87906F45025C87906F49025C874D
:105BDC00906F4D025C87906F51025C87906F5502FD
:105BEC005C87906F59025C87906F5D025C87906F49
:105BFC0061025C87906F65025C87906F69025C87BD
:105C0C00906F6D025C87906F71025C87906F75026C
:105C1C005C87906F79025C87906F7D025C87906FD8
:105C2C0081025C87906F85025C87906F89025C872C
:105C3C00906F8D025C87906F91025C87906F9502DC
:105C4C005C87906F99025C87906F9D025C87906F68
:105C5C00A1025C87906FA5025C87906FA9025C879C
:105C6C00906FAD025C87906FB1025C87906FB5024C
:105C7C005C87906FB9025C87906FBD05A290005E47
:105C8C007B04129176229002B6E070037B002230E6
:105C9C00550A900172E06004126BA42290018AE014
:105CAC00B41906125D04025CE49004B8E0F57C9033
:105CBC0004B7E004B57C15900193E0B402069001A2
:105CCC004D7400F09004B77400025CDA50E9F09067
:105CDC0004B7E0125F1DE0FB9004B9F0123445905C
:105CEC000171F0900172EAF0900175E0B2E0F012EF
:105CFC006BB59004B9E0FB229004B8E0126C7912F9
:105D0C005F1DE0FB229002B6E0700122128E8290A1
:105D1C00018AE01475F003A4905D2873025D730290
:105D2C005E0F025E62025E91025EE8025F38025F05
:105D3C0070025FB5025FFA0260110260A50260E6B4
:105D4C0002612402616C0261AC0261E50261FF0236
:105D5C0062190262360262E80263510263DA02647B
:105D6C000002640A02644C125D7722125D7E125DA1
:105D7C00CB229002B6E0120D3EFA7BFF7C00900223
:105D8C00B705A290022A128C96E0A30B30E7FA0515
:105D9C00A2EBF0A305A20CDAF0EC9004B8F0FF2211
:105DAC009004B8E09002B78582378583387837F550
:105DBC003B753C00793B12036E86820886832290E9
:105DCC00018CE0F57C157C7E01B4010122125DE0B2
:105DDC00D57CFA22EE75F00CA4FD0E125DACEFFB37
:105DEC007C0005A29002B7E0A32D05A2F0A305A2AA
:105DFC000CECB4FF059004B8F022DBEB9004B8E097
:105E0C002CF022125D77125E19125E32229004B8C9
:105E1C00E0FB9003B705A2EB14125F1DE005A2F0A6
:105E2C00A305A2DBF2229004B8E0FB9002B705A216
:105E3C009003B7E0A305A2F0A305A2DBF622900421
:105E4C00B8E0FB9003B705A29002B7E0A305A2F05F
:105E5C00A305A2DBF622125D77125E19125E6C228C
:0E5E6C009004B8E0FC1414FBEC125F1D05A2BC
:105E7A009003B87C00E0A305A2F0A305A20CDBF511
:105E8A009004B8E02CF022125D779004B8E0B402D6
:105E9A00012240FD125E19125EA8125E322290049F
:105EAA00B8E0FC1414FBEC125ECD05A29002B87C9B
:105EBA0000E0A305A2F0A305A20CDBF59004B8E06C
:105ECA002CF0229003B78582378583387837F53BE3
:105EDA00753C00793B12036E868208868322125D26
:105EEA00779004B8E0B402012240FD125E19125EF6
:105EFA00FC229004B8E0FB125F1D05A29003B7E0F4
:105F0A00A305A2F0A305A2DBF69004B8E075F0029F
:105F1A00A4F0229002B78582378583387837F53B1B
:105F2A00753C00793B12036E868208868322125DD5
:105F3A00779004B8E0B402012240FD125E19125FA4
:105F4A004F125E32229004B8E0FB125ECD05A29099
:105F5A0002B7E0A305A2F0A305A2DBF69004B8E01D
:105F6A0075F002A4F022125D779004B8E0B4020141
:105F7A002240FD125F84125E32229004B8E0FB14C4
:105F8A00FC7D009002B705A29003B705A2ED125F4F
:105F9A001D0DE005A2F0A305A2EC125F1D1CE00591
:105FAA00A2F0A31BEB700122DBE122125D779004C1
:105FBA00B8E0B402012240FD125FC9125E3222909B
:105FCA0004B8E0FB14FC7D009002B705A29003B769
:105FDA0005A2EC125F1D1CE005A2F0A305A2ED12BA
:105FEA005F1D0DE005A2F0A31BEB700122DBE1228D
:105FFA00125D779004B8E0B402012240FD125F847A
:10600A00126064125E3222125D779004B8E0B40224
:10601A00012240FD125FC9126028125E32229004EA
:10602A00B8E0FEFB14FC7D009002B705A21260A046
:10603A0005A2ED125F1D0DE005A2F00EA305A2EC6C
:10604A00125F1D1CE005A2F00EA31BEB7004026098
:10605A005E22DBDC9004B8EEF0229004B8E0FEFB8E
:10606A0014FC7D009002B705A21260A005A2EC12F2
:10607A005F1D1CE005A2F00EA305A2ED125F1D0D27
:10608A00E005A2F00EA31BEB700402609A22DBDC8F
:10609A009004B8EEF022EB125ECD22125D779004E6
:1060AA00B8E0B402012240FD1260B9125E322290B9
:1060BA0004B8E014FB7C007D019002B7E0FF05A262
:1060CA009003B7EFF00CA305A2ED125F1D0DE005DA
:1060DA00A2F00CA3DBED9004B8ECF022125D7790ED
:1060EA0004B8E0B402012240FD1260FA125E3222C4
:1060FA009004B8E014FB7C009002B7E0FF05A29080
:10610A0003B7EFF00CA305A2EB125F1DE005A2F0A6
:10611A000CA3DBEE9004B8ECF022125D779004B881
:10612A00E0B402012240FD125E19125E6C12613E59
:10613A00125E32229004B8E01414FB7C007D0190B8
:10614A0002B7E0FF05A29003B7EFF00CA305A2ED9A
:10615A00125F1D0DE005A2F00CA3DBED9004B8EC74
:10616A00F022125D779004B8E0B402012240FD12D9
:10617A005E19125E6C12613E126189125E322290C1
:10618A0004B8E075F00284FCFB9003B705A2EC1298
:10619A005ECDE0FF05A2E0CFF0A305A2EFF0A3DBFE
:1061AA00F122125D779004B8E0B401012240FD1299
:1061BA0061C0125E32229004B8E0FB9003B705A2D8
:1061CA009002B7E0A305A2F0A3240CF0A305A2DB7A
:1061DA00F29004B8E075F002A4F022125D77900400
:0E61EA00B8E0B401012240FD125E19125E32CF
:1061F8001261C0125E3222125D779004B8E0B401D9
:10620800012240FD125E19125E6C1261C0125E32EC
:1062180022125D779004B8E0B401012240FD125EBD
:1062280019125E6C1261C0126189125E322212620A
:10623800599004B8E0B4020A125E4A1262A8125ECB
:10624800322240F41262901262631262A8125E3225
:10625800229002B6E0120D2B025D859004B8E0FB97
:10626800FDFF7E007C009003B705A29002B7E0A373
:1062780005A2F0A305A20CDBF50EEDFBEE125F1DE7
:10628800DFEC9004B8ECF0229004B8E0FB125F1D3C
:1062980005A29002B7E0A305A2F0A305A2DBF622AF
:1062A80090018CE014700122FF7D009004B8126206
:1062B800C39004B8E00D8DF0A4F022E0FCFB0DECD7
:1062C800FB8DF0A4125ECD05A29003B7ED75F00C1E
:1062D800A4FEE02EA305A2F0A305A2DBEFDFDF22D8
:1062E8001262599004B8E0B4020A125E4A126311AD
:1062F800125E322240F4125E19125E32126290125D
:106308006263126311125E322290018CE0147001F4
:1063180022FF7D009004B812632C9004B8E00D8D24
:10632800F0A4F022E0FCFB0DECFB8DF0A4125ECD96
:1063380005A29003B7EF75F00CA4FEE02EA305A20A
:10634800F0A305A2DBEFDFDF22125D7E9004B8E048
:10635800B4020A125E4A1262A8125E322240F41295
:1063680063711262A8125E32229004B8E0FB7C00CE
:106378009003B705A29002B7E0A305A2F00CA3050D
:10638800A2DBF59004B8E014FB9002B8E0A305A2E4
:10639800F00CA305A2DBF59002B7E0240CA305A23C
:1063A800F00CA305A29004B8E01414FB9002B9E025
:1063B800A305A2F00CA305A2DBF57B029002B7E0CF
:1063C800240CA305A2F00CA305A2DBF39004B8ECFF
:1063D800F022125D7E9004B8E0B4020A125E19122F
:1063E8006311125E322240F4126371125E32125E41
:1063F80019126311125E32221264141262A8125E1C
:1064080032221264141262A81264332290021DE030
:106418007001229004B8F0FB9003B705A290020522
:10642800E0A305A2F0A305A2DBF6229004B8E0FBE6
:106438009002B705A2EB14125ECDE005A2F0A30509
:10644800A2DBF222125D772290056BE070037B00DD
:106458002230560A900174E06004126BD222900137
:10646800A1E0B419061264C20264A290066DE0F5B8
:106478007C90066CE004B57C159001AAE0B4020695
:106488009001507400F090066C740002649850E912
:10649800F090066CE01266B7E0FB90066EF0123DD5
:1064A80024900173F0900174EAF0900175E0B2E174
:1064B800F0126BE390066EE0FB2290066DE0126C22
:1064C800791266B7E0FB2290056BE0700122128F0B
:1064D800349001A1E01475F003A49064E67302659A
:1064E800310265C40266170266460266820266D2F7
:1064F80002670A02674F0267940267AB02683A02B2
:10650800687B0268B902690102692502695E02694D
:10651800780269920269AF026A61026AA5026B2E6B
:10652800026B54026B5E026BA01265352212653C49
:106538001265892290056BE0120D3EFA7BFF7C0004
:1065480090056C05A29004DF128CA4E0A30B30E741
:10655800FA05A2EBF0A305A20CDAF0EC90066DF0B8
:0E656800FF2290066DE090056C8582378583DA
:10657600387837F53B753C00793B12036E86820806
:106586008683229001A3E0F57C157C7E01B401018F
:106596002212659ED57CFA22EE75F00CA4FD0E1231
:1065A600656AEFFB7C0005A290056CE0A32D05A2B1
:1065B600F0A305A20CDBF490066DE02CF022126528
:1065C600351265CE1265E72290066DE0FB9003B7A3
:1065D60005A2EB141266B7E005A2F0A305A2DBF252
:1065E6002290066DE0FB90056C05A29003B7E0A330
:1065F60005A2F0A305A2DBF62290066DE0FB900350
:10660600B705A290056CE0A305A2F0A305A2DBF6F0
:10661600221265351265CE1266212290066DE0FCC7
:106626001414FBEC1266B705A29003B87C00E0A335
:1066360005A2F0A305A20CDBF590066DE02CF02276
:1066460012653590066DE0B402012240FD1265CE5A
:1066560012665D1265E72290066DE0FC1414FBECF1
:10666600125ECD05A290056D7C00E0A305A2F0A305
:1066760005A20CDBF590066DE02CF0221265359034
:10668600066DE0B402012240FD1265CE1266962226
:1066960090066DE0FB1266B705A29003B7E0A3056E
:1066A600A2F0A305A2DBF690066DE075F002A4F059
:1066B6002290056C8582378583387837F53B753CA3
:1066C60000793B12036E8682088683221265359016
:1066D600066DE0B402012240FD1265CE1266E91293
:1066E60065E72290066DE0FB125ECD05A290056C73
:1066F600E0A305A2F0A305A2DBF690066DE075F017
:1067060002A4F02212653590066DE0B40201224023
:10671600FD12671E1265E72290066DE0FB14FC7DF4
:106726000090056C05A29003B705A2ED1266B70DA1
:10673600E005A2F0A305A2EC1266B71CE005A2F0E4
:10674600A31BEB700122DBE12212653590066DE09A
:10675600B402012240FD1267631265E72290066DBE
:10676600E0FB14FC7D0090056C05A29003B705A222
:10677600EC1266B71CE005A2F0A305A2ED1266B7FF
:106786000DE005A2F0A31BEB700122DBE1221265EE
:106796003590066DE0B402012240FD12671E1267B5
:1067A600FE1265E72212653590066DE0B4020122FD
:1067B60040FD1267631267C21265E72290066DE01C
:1067C600FEFB14FC7D0090056C05A21260A005A2DC
:1067D600ED1266B70DE005A2F00EA305A2EC126657
:1067E600B71CE005A2F00EA31BEB70040267F822AB
:1067F600DBDC90066DEEF02290066DE0FEFB14FCED
:106806007D0090056C05A21260A005A2EC1266B789
:106816001CE005A2F00EA305A2ED1266B70DE00579
:10682600A2F00EA31BEB700402683422DBDC900698
:106836006DEEF02212653590066DE0B4020122403D
:10684600FD12684E1265E72290066DE014FB7C008F
:106856007D0190056CE0FF05A29003B7EFF00CA355
:1068660005A2ED1266B70DE005A2F00CA3DBED90D4
:10687600066DECF02212653590066DE0B402012239
:1068860040FD12688F1265E72290066DE014FB7CCE
:106896000090056CE0FF05A29003B7EFF00CA3058E
:1068A600A2EB1266B7E005A2F00CA3DBEE90066D34
:1068B600ECF02212653590066DE0B402012240FD2F
:1068C6001265CE1266211268D31265E72290066D14
:1068D600E01414FB7C007D0190056CE0FF05A2909E
:0E68E60003B7EFF00CA305A2ED1266B70DE0AC
:1068F40005A2F00CA3DBED90066DECF022126535D9
:1069040090066DE0B402012240FD1265CE126621AC
:106914001268D312691E1265E72290066D12618C0B
:106924002212653590066DE0B401012240FD126922
:10693400391265E72290066DE0FB9003B705A2903B
:10694400056CE0A305A2F0A3240CF0A305A2DBF2DE
:1069540090066DE075F002A4F02212653590066D84
:10696400E0B401012240FD1265CE1265E7126939D7
:106974001265E72212653590066DE0B402012240EB
:10698400FD1265CE1266211269391265E72212657D
:106994003590066DE0B402012240FD1265CE126608
:1069A4002112693912691E1265E7221269D2900612
:1069B4006DE0B4020A1265FF126A211265E72240F3
:1069C400F4126A091269DC1262A81265E7229005C2
:1069D4006BE0120D2B02654390066DE0FBFDFF7E1C
:1069E400007C009003B705A290056CE0A305A2F01B
:1069F400A305A20CDBF50EEDFBEE1266B7DFEC90FF
:106A0400066DECF02290066DE0FB1266B705A290CD
:106A1400056CE0A305A2F0A305A2DBF6229001A376
:106A2400E014700122FF7D0090066D126A3C90060E
:106A34006DE00D8DF0A4F022E0FCFB0DECFB8DF07D
:106A4400A4125ECD05A29003B7ED75F00CA4FEE090
:106A54002EA305A2F0A305A2DBEFDFDF221269D289
:106A640090066DE0B4020A1265FF126A8A1265E7A5
:106A74002240F41265CE1265E7126A091269DC122B
:106A84006A8A1265E7229001A3E014700122FF7D57
:106A94000090066D12632C90066DE00D8DF0A4F04D
:106AA4002212653C90066DE0B4020A1265FF126A78
:106AB400211265E72240F4126AC5126A211265E7C1
:106AC4002290066DE0FB7C009003B705A290056C54
:106AD400E0A305A2F00CA305A2DBF590066DE0147B
:106AE400FB90056DE0A305A2F00CA305A2DBF590D5
:106AF400056CE0240CA305A2F00CA305A290066D7E
:106B0400E01414FB90056EE0A305A2F00CA305A20B
:106B1400DBF57B0290056CE0240CA305A2F00CA32A
:106B240005A2DBF390066DECF02212653C90066D35
:106B3400E0B4020A1265CE126A8A1265E72240F4B2
:106B4400126AC51265E71265CE126A8A1265E722D7
:106B5400126B68126A211265E722126B68126A21AD
:106B6400126B87229004D2E070012290066DF0FB34
:106B74009003B705A29004BAE0A305A2F0A305A26E
:106B8400DBF62290066DE0FB90056C05A2EB141277
:106B94005ECDE005A2F0A305A2DBF2221265352248
:106BA4009004B9E0FB900171E014F0600122C25539
:106BB40022BA0103D25522BA020720E00122D2559B
:106BC40022BA030720E003D2552222C2552290069E
:106BD4006EE0FB900173E014F0600122C25622BA09
:106BE4000103D25622BA020720E10122D25622BA68
:106BF400030720E103D2562222C25622900072E0FB
:106C040004B410027400F0900062A98229F582E0B5
:106C140022900076E0FA900073E004B40F0274FF4F
:106C2400F0906CED932A900076F0900075E004B437
:106C340010027400F0F9900076E0FA900062E582A8
:106C440029F582EAF022900076E0FA900074E004DC
:106C5400B4110274FFF0906CFC932A900076F01249
:0E6C64006C2E22126C0054016008126C005459
:106C72001F246022747F22F974FF89F084F5F012D8
:106C82006C008422126C0075F0208422126C007554
:106C9200F03384240122126C0075F0208424012236
:106CA200126C0075F03F84240122126C0075F033DF
:106CB20084240322126C0075F0108422126C007579
:106CC200F01F8422126C0075F02084F8126C00759B
:106CD200F03F842822126C00540175F00CA4221299
:106CE2006C0075F0558475F00CA422037F2C0C0106
:106CF20005712133E6FF0B576818BD09A60D004B3D
:106D02005D263585B196114093C8D3464C414D4519
:106D1200204152504547474941544F52204D4F441C
:106D2200554C45204555524F205241434B20564524
:106D32005253494F4E202D20323031352056455284
:106D420053494F4E20312E30352028632962792055
:106D5200616D70657265204620204C202041202004
:106D62004D20204520204152504547474941544F2C
:106D7200522032303133202056455253494F4E2053
:106D8200312E303720202020286329323031332D14
:106D9200323031352020496E697420616C6C204498
:106DA200617461203F204F4B202020202020202092
:106DB2002020204E4F2020506C6561736520776142
:106DC2006974202120202020202020202020202023
:106DD20020202020202020202020202020202020B1
:106DE20020202020202020202020202020202020A1
:106DF2002020202020206F66664152502020204211
:106E0200415353202043484F5244205343414C4561
:106E1200204D4944492020534554555020584F5540
:106E2200543A204C49535420205341564520205077
:106E32004C41594C49535420444154412020206D27
:106E42006972726F72656420536571426173736D0A
:106E52006972726F72656420536571204172706D40
:106E62006972726F7265642053657120582D313AD0
:106E720041203A4220543A633A733A4C49535420DF
:106E820020202020204C656E6768744C313220230C
:106E920043206350303120417365715430302020DB
:106EA200442073553136203473657141706F7241DD
:106EB2006E74724173657141436C6B4164756F41CD
:106EC20074726941646F7441676174563132375626
:106ED200726E643173657131436C6B3164756F31FD
:106EE20074726931646F74316761743273657132BF
:106EF200436C6B3264756F3274726932646F7432D0
:106F02006761743373657133436C6B3364756F33CC
:106F120074726933646F7433676174347365713486
:106F2200436C6B3464756F3474726934646F743497
:106F3200676174546D706F42706F72426E74724208
:106F420073657142436C6B4264756F42747269423D
:106F5200646F74426761745631323756726E6435AB
:106F620073657135436C6B3564756F357472693551
:106F7200646F74356761743673657136436C6B3652
:106F820064756F3674726936646F7436676174370C
:106F920073657137436C6B3764756F377472693719
:106FA200646F74376761743873657138436C6B381A
:106FB20064756F3874726938646F74386761743ECF
:106FC2004120203E4220203E414220582D3120586F
:106FD2002D3220582D3320582D3420582D3520584D
:0E6FE2002D3620582D3720582D3820202053D2
:106FF000455454494E47533E43686F72643A553086
:10700000313E5363616C653A553031413E534551D1
:107010003136553031423E5345513136553031507D
:107020007265737320204B45594E4F5445202120E3
:107030002053544F52414745204F4B2021202020C0
:1070400020202020204D4F44454E4F54455245505E
:10705000454154202020202052414E4745202020E9
:107060002020474C494445205345513A3136503051
:10707000312020202020434C4F434B202020202033
:107080002047415445202056454C4F4349545920F0
:10709000534551552D4D4F44454C4F4F502D524562
:1070A00053455420204F55542D474154452020200E
:1070B000204F55542D4356584F55543A31203136B0
:1070C0003A536571503031424153532020203136BC
:1070D0003A536571503031202020202054454D50C6
:1070E0004F20202020202053594E43524543562004
:1070F000434C4F434B53454E4420434C4F434B204E
:1071000052454356204348414E202041525020438F
:1071100048414E2042415353204348414E43484F3B
:107120005244204348414E582D4F55542043484126
:107130004E65787465726E204D696469436C6F6347
:107140006B20202020696E7465726E20436C6F6323
:107150006B43686F72642054726967676572204977
:107160006E4152502B42415353205472696720495B
:107170006E6E6F726D616C202068616C66202020DD
:107180006F666620555345522D3120494E20555388
:1071900045522D3220494E2054554E452D4D4F44D9
:1071A000455365742043562D4F5554733A202B3167
:1071B000564172703A20582D313A20582D323A20DB
:1071C000582D333A20582D343A20426173733A587F
:1071D0002D353A20582D363A20582D373A20582D43
:1071E000383A20202020202020474C494445204E7A
:1071F0004F54455245504541542020205345515548
:10720000454E43452020434C4F434B20414C4C209E
:1072100020434C4F434B2044554F2020434C4F4379
:107220004B205452492020434C4F434B20444F5451
:10723000202020202020204741544556454C4F20F7
:10724000312E2E31323756454C4F20416363526EFA
:107250006420202020555345522D312020202055D8
:107260005345522D32436C61737369633A20202079
:107270002020207570436C61737369633A2020206D
:1072800020646F776E436C61737369633A20207575
:1072900070646F776E436C61737369633A20206426
:1072A0006F776E7570436F70793A2020202075706B
:1072B0002B646F776E436F70793A20202020646FC3
:1072C000776E2B757050696E67506F6E673A20202D
:1072D000202020757050696E67506F6E673A2020CD
:1072E00020646F776E50696E67506F6E673A2075D5
:1072F00070646F776E50696E67506F6E673A206486
:107300006F776E757046697420526F6F743A2020E3
:10731000202020757046697420526F6F743A2020C7
:1073200020646F776E46697420526F6F743A2075CF
:1073300070646F776E46697420526F6F743A206480
:107340006F776E7570466974204F637461763A206A
:107350002020207570466974204F637461763A204E
:0E73600020646F776E466974204F6374617607
:10736E003A7570646F776E466974204F63746176F8
:10737E003A646F776E7570536B69703A20202020D7
:10738E0020202020207570536B69703A2020202019
:10739E00202020646F776E496E76657273696F6E0A
:1073AE003A202020207570496E76657273696F6E73
:1073BE003A2020646F776E4F7264657265643A206E
:1073CE00202020202075704F7264657265643A200B
:1073DE00202020646F776E20202020202020202067
:1073EE002052616E646F6D202020202020202020EE
:1073FE00202020206F6666202020202020202020A4
:10740E00656163683A2031416C7465726E617465B2
:10741E00203173743A2031416C7465726E617465FB
:10742E0020326E643A20312020202020202032206D
:10743E006F637461766573202020206D6178696DAD
:10744E00616C3A20313238506F7274616D2E54690E
:10745E006D653A20313237202020207374657020FC
:10746E0062792073746570202020202020202063F4
:10747E006F6D62696E6564206174206172706567FC
:10748E0067696F20656E6420617420736571756520
:10749E006E636520656E64696E7465726E436C6FA3
:1074AE00636B2F4D494449547269676765722D4964
:1074BE006E2020312F3136547269676765722D49FF
:1074CE006E205469636B73547269676765722D49D8
:1074DE006E205374657073202053657175656E63ED
:1074EE0065284761746529202020526573657420D4
:1074FE007065722042617220204172706567676903
:10750E006F2052657365744F75742D333A20205673
:10751E00656C6F636974794F75742D333A43686F78
:10752E007264206E6F74654F75742D343A20205638
:10753E00656C6F636974794F75742D343A43686F57
:10754E007264206E6F746520202020202066697280
:10755E007374206E6F7465202020202020206C61B3
:10756E007374206E6F7465416363656E743A206543
:10757E0061636820326E64416363656E743A2065A0
:10758E0061636820337468416363656E743A206585
:10759E0061636820347468416363656E743A206574
:1075AE0061636820357468416363656E743A206563
:1075BE0061636820367468416363656E743A206552
:1075CE0061636820377468416363656E743A206541
:1075DE0061636820387468416363656E743A206530
:1075EE006163682039746852616E646F6D3A202051
:1075FE0020312E2E31323752616E646F6D3A20205B
:10760E0036342E2E31323752616E646F6D3A202031
:10761E0037362E2E31323752616E646F6D3A20201E
:10762E0039352E2E31323752616E646F6D3A2031FC
:10763E0031322E2E31323752616E646F6D3A202008
:10764E00666F726D756C61202020202020202066D0
:10765E0069783A2031323731205469636B3A2031E0
:10766E002F36342074726933205469636B733A2059
:10767E00202020312F333236205469636B733A2029
:10768E00202020312F313631325469636B733A200A
:10769E0020202020312F3832345469636B733A2006
:1076AE0020202020312F3434385469636B733A20F4
:1076BE0020202020312F3239365469636B733A20E3
:1076CE002020312062617232205469636B733A312B
:0E76DE002F33322074726934205469636B7349
:1076EC003A312F31362074726938205469636B73C8
:1076FC003A20312F382074726931365469636B73B8
:10770C003A20312F342074726933325469636B73AD
:10771C003A20312F322074726936345469636B739A
:10772C003A20312F312074726939205469636B739C
:10773C003A312F313620646F7431385469636B736E
:10774C003A20312F3820646F7433365469636B736D
:10775C003A20312F3420646F7437325469636B7361
:10776C003A20312F3220646F74204E4F54204156F2
:10777C0041494C41424C4520210103060C18306014
:10778C0002040810204009122448202020202061E7
:10779C006461707465643A20203361646170742E86
:1077AC0072616E646F6D3A312D3561646170742E47
:1077BC0072616E646F6D3A312D3861646170742E34
:1077CC0072616E646F6D3A332D38202066697820B3
:1077DC0072616E646F6D3A20343820202020616312
:1077EC0063656E7420206C6F6E67202020206163AF
:1077FC0063656E742073686F7274202020202020C3
:10780C002020206669783A203938010101010101F4
:10781C00010201010102020202030101020304043C
:10782C00050601020406080A0B0C0104080C1014CE
:10783C0017180108101820282E3001102030405045
:10784C005C60010101010202020301010202020358
:10785C0003040102030405060708010204080A0CCC
:10786C000E100104081014181C20010810202830D8
:10787C0038400102030405060809010306080A0C36
:10788C00101201060C1014182024010C182028309A
:10789C0040480110203040505FC04B45594E4F546A
:1078AC00453A2020432343204423442045204623AB
:1078BC004620472347204123412042234330206D5B
:1078CC00616A6F72203720202020520000FFFF8059
:1078DC000080808888AAAA0808141422225555EE24
:1078EC00EEE38EE388C30CDB6F9999BABAAB5ADB23
:1078FC006EDB6AADADD6D6AAD5A9A9ABABDADA9256
:10790C0049BBBBAA9AAAD7CAE2A9A9FFF08000AAD0
:10791C00A0AD60A940AD502950AB502A50ABC0A2CD
:10792C0040B2C0BEF09200B6A0A0A0249002A09AD3
:10793C000089800920BBE0A990A9E0BAE0EAC092D6
:10794C0040A280B2C0B6D0FEA0F8008000C000E01B
:10795C0000F000A800B000D000FE008000AA00D803
:10796C0000E000EC00F400D400FF808000AA80DB73
:10797C0000ED00F700B680CA80FFC08000AA808AA4
:10798C0080EA80A500B580F580FFE08000AAA0D237
:10799C0080EAC0F540F780E740FFF88000AAA8DB3A
:1079AC0060E770BDA0F7B0F9F0FFFC8000AAA8DB7F
:1079BC0068FDF8EDD8FAB0D49CFFFE8000AAAAE9C5
:1079CC00DCEEECF5DABDDCFAB2030004070C0400C3
:1079DC00040709040004070B040004060B0400044C
:1079EC00080B040002040704000405070400040744
:1079FC000E030003060C040004070A040004060A24
:107A0C00030005070C0400020507040002050A0325
:107A1C000003070C0400030709040003070A040011
:107A2C0003060A040003080A040002030704000307
:107A3C000507030003070E040003060904000306F0
:107A4C000A030004080C040004080A030002070CD3
:0E7A5C00040005070A0300050A0C02000000E2
:107A6A000002000100000200020000020003000000
:107A7A0002000400000200050000020006000002E5
:107A8A0000070000020008000002000900000200CE
:107A9A000A000002000B000002000C0000020000B5
:107AAA0000000200010000020002000002000300C0
:107ABA0000020004000002000500000200060000A7
:107ACA00020007000002000800000200090000028C
:107ADA00000A000002000B000002000C0000202037
:107AEA002020202020202020204D616A6F72202033
:107AFA00202020202020204D616A6F72203620200D
:107B0A00202020202020204D616A6F7220372020FB
:107B1A0020202020204D616A6F7220376235202094
:107B2A0020202020204D616A6F72203723352020C3
:107B3A002020202020202020206164642032202060
:107B4A00202020202020202020616464203420204E
:107B5A002020202020202020206164642039202039
:107B6A002020202044696D696E697368656420204D
:107B7A0020202020202020202020202020372020E4
:107B8A00202020202020202020202037623520207D
:107B9A0020202020202020202073757320342020CC
:107BAA0020202073757320342073757320322020AF
:107BBA002020202050656E7461746F6E69632020E6
:107BCA002020202020202020204D696E6F72202046
:107BDA00202020202020204D696E6F722036202020
:107BEA00202020202020204D696E6F72203720200F
:107BFA00202020204D696E6F7220372062352020A8
:107C0A00202020204D696E6F7220372023352020D6
:107C1A002020204D696E6F7220616464203220201A
:107C2A002020204D696E6F72206164642034202008
:107C3A002020204D696E6F722061646420392020F3
:107C4A00202044696D696E69736865642037202055
:107C5A002020202068616C662064696D203720200E
:107C6A0020202020204175676D656E746564202090
:107C7A0020202020202020202020372023352020CB
:107C8A0020202020202020202073757320322020DD
:107C9A0020202020202020372073757320342020B4
:107CAA0020202020202020466F75727468732020BF
:107CBA0020496E74657276616C2020302D30202048
:107CCA0020496E74657276616C2020302D31202037
:107CDA0020496E74657276616C2020302D32202026
:107CEA0020496E74657276616C2020302D33202015
:107CFA0020496E74657276616C2020302D34202004
:107D0A0020496E74657276616C2020302D352020F2
:107D1A0020496E74657276616C2020302D362020E1
:107D2A0020496E74657276616C2020302D372020D0
:107D3A0020496E74657276616C2020302D382020BF
:107D4A0020496E74657276616C2020302D392020AE
:107D5A0020496E74657276616C20302D3130202096
:107D6A0020496E74657276616C20302D3131202085
:107D7A0020496E74657276616C20302D3132202074
:107D8A0020202020757365722063686F7264080072
:107D9A000305070206080B00000000060004070896
:107DAA0001050000000000000500030708010000AB
:107DBA000000000000060003070A04090000000092
:107DCA000000060003050A0607000000000000077D
:0E7DDA000004070B01050800000000000C006B
:107DE80003070A010204050608090B050002040737
:107DF8000900000000000000070004070B01050847
:107E08000000000000070004080B01060A0000003B
:107E18000000050005070A02000000000000000736
:107E28000004070A02050800000000000700040714
:107E38000A0306090000000000070003070B0206FA
:107E48000800000000000500030708020000000009
:107E5800000000050005060A0100000000000000FF
:107E680005000507080100000000000000050005E6
:107E7800070A0100000000000000050003070A05CA
:107E880000000000000000050005070A02000000CD
:107E980000000000050004070902000000000000BF
:107EA80000070004060A0205080000000000070099
:107EB80003060A0104080000000000070004070A7E
:107EC8000206080000000000070004070902050B6D
:107ED8000000000000040004070900000000000082
:107EE8000000040004070B0000000000000000046C
:107EF8000004060A00000000000000000700030755
:107F08000A02050800000000000400030709000039
:107F1800000000000000040003070A000000000041
:107F2800000000070003070B02050800000000001E
:107F3800070004070B020509000000000007000203
:107F4800060A0305090000000000070003070A01EC
:107F580005080000000000070004070B02060900DE
:107F680000000000070004070A02050900000000DD
:107F7800070003070A0205080000000000070003C5
:107F8800060A0105080000000000070003070901B0
:107F9800050B0000000000070003070B010508009F
:107FA800000000000900030709020406080B00008E
:107FB80000080004070A0103060900000000070082
:107FC80004060A0105090000000000070004070A6A
:107FD8000206090000000000050003070801000070
:107FE800000000000005000507090200000000006D
:107FF8000000050004070902000000000000000559
:10800800000305070A000000000000000500040640
:108018000A0200000000000000070004080A010529
:1080280007000000000008000306090104070A0011
:10803800000000060004080A020600000000000014
:10804800070004080B02060A000000000020202098
:108058002020202020416C67657269616E202020F5
:108068002020202020204172616269616E2020203A
:1080780020202042616C696E657369616E20202042
:108088002020426C756573206D616A6F7220202014
:108098002020426C756573206D696E6F72202020F8
:1080A8002020202042797A616E74696E6520202034
:1080B800202020204368726F6D617469632020203E
:1080C8002020202020446961746F6E696320446F0A
:1080D80075626C65204861726D6F6E69632020203F
:1080E80020202020456E69676D6174696320202017
:1080F8002020202020456779707469616E20202037
:108108002020202048696E64757374616E2048755C
:108118006E67617269616E206D616A6F7220487561
:108128006E67617269616E206D696E6F724A617007
:10813800616E3A2068697261796F7368694A617023
:10814800616E3A697761746F796F7368694A6170B3
:0E815800616E3A6B756D6F69796F7368694A75
:108166006170616E3A2020202020696E73656E4A28
:108176006170616E3A2020202020796F73656E4A07
:108186006170616E3A2020726974737573656E4A08
:108196006170616E3A2020202072796F73656E20BF
:1081A60020206D616A6F72204C6F637269616E2068
:1081B60020207375706572204C6F637269616E2042
:1081C6002020204C796469616E206D696E6F722083
:1081D600202020202020202020204D616A6F722040
:1081E60020202020202020204D616A6F722036201A
:1081F60020202020202020204D616A6F7220372009
:1082060020202020204D616A6F72203720623520A1
:10821600202020202020202020204D696E6F7220F3
:1082260020202020202020204D696E6F72203620CD
:1082360020202020202020204D696E6F72203720BC
:10824600204D696E6F72206861726D6F6E69634D45
:108256006F64653A2020202020496F6E69616E4D5B
:108266006F64653A2020202020446F7269616E4D4C
:108276006F64653A202020506872796769616E4D97
:108286006F64653A20202020204C796469616E4D28
:108296006F64653A204D69786F6C796469616E4DDB
:1082A6006F64653A2020202041656F6C69616E4DD0
:1082B6006F64653A202020204C6F637269616E4EB0
:1082C6006561706F6C6974616E206D616A6F724E64
:1082D6006561706F6C6974616E206D696E6F722076
:1082E6002020202020204E696E6520546F6E652068
:1082F6002020202020204F637461746F6E696320F4
:10830600202020202020204F7269656E74616C2029
:10831600202020202020204F766572746F6E652005
:108326002020202020202020202050656C6F6720F0
:10833600202020202050656E7461746F6E69636D15
:10834600616A6F722050656E7461746F6E69636DD9
:10835600696E6F722050656E7461746F6E6963200A
:10836600202020202050726F6D657468657573201B
:1083760020202020202020205370616E6973682001
:108386002020202053796D6D6574726963616C20BD
:1083960020202020202057686F6C65746F6E656CF6
:1083A600656164696E6757686F6C65746F6E65208A
:1083B600202020202075736572207363616C65032D
:1083C600000407000000000000000000030004078E
:1083D6000000000000000000000700040702050975
:1083E6000B00000000000101010101010101010172
:1083F60001011E1E1E1E1E1E1E1E1E1E1E1E01010B
:108406000101010101010101010101010101010156
:108416000101010101010CFF00FF01FF02FF03FF43
:1084260004FF05FF06FF07FF08FF09FF0AFF0BFF12
:108436000CFF0DFF0EFF0FFF10FF11FF12FF13FFC2
:1084460014FF15FF16FF17FF18FF19FF1AFF1BFF72
:108456001CFF1DFF1EFF1FC2A5C2A4C295C2A3E535
:108466005020160274FF7F083392A6D2A3C2A3DF60
:10847600F7B2A50000C2A5E55120160274FF7908DF
:108486003392A6C2A3D2A3D9F7D2A40000C2A422D3
:10849600C2A6D2A67908C2A3A2A733D2A3D9F7F55A
:1084A6006AC2A6D2A67908C2A3A28033D2A3D9F7FC
:1084B600F56B2290017CE0B403030284CD50FB905F
:1084C600017EE0B405012290017CE0B4070122B4EC
:0E84D600080122E56B20E50122E56B20E6019E
:1084E4002212850A12858D1286101286931287161F
:1084F40012879912881C12889F1289221289A51248
:108504008A28128AAB22E56B30E10DC217202314AE
:10851400D223128559D23222C223201707D217122E
:108524008529D2322220520620531A028539128517
:10853400391285492290022A128CB2E0B2E7F07F08
:1085440000128ECE229004DF128CDBE0B2E7F07FC3
:1085540000128ED92220520620531C0285691285EE
:108564006912857B22203A2090022A128CB2740070
:10857400F07F00128E4A22203B0E9004DF128CDB27
:108584007400F07F00128EFC22E56B30E20DC218FD
:10859400202414D2241285DCD23222C224201807CB
:1085A400D2181285ACD2322220520620531A0285E8
:1085B400BC1285BC1285CC2290022B128CB2E0B284
:1085C400E7F07F01128ECE229004E0128CDBE0B241
:1085D400E7F07F01128ED92220520620531C028517
:1085E400EC1285EC1285FE22203A2090022B128C8C
:1085F400B27400F07F01128E4A22203B0E9004E0F8
:10860400128CDB7400F07F01128EFC22E56B30E3E8
:108614000DC219202514D22512865FD23222C2251A
:10862400201907D21912862FD23222205206205343
:108634001A02863F12863F12864F2290022C128C19
:10864400B2E0B2E7F07F02128ECE229004E1128CE7
:10865400DBE0B2E7F07F02128ED9222052062053CB
:108664001C02866F12866F12868122203A209002A5
:108674002C128CB27400F07F02128E4A22203B0E20
:108684009004E1128CDB7400F07F02128EFC22E570
:108694006A30E00DC21A202614D2261286E2D232A3
:1086A40022C226201A07D21A1286B2D232222052AD
:1086B4000620531A0286C21286C21286D222900261
:1086C4002D128CB2E0B2E7F07F03128ECE2290041A
:1086D400E2128CDBE0B2E7F07F03128ED922205243
:1086E4000620531C0286F21286F212870422203AD4
:1086F4002090022D128CB27400F07F03128E4A2255
:10870400203B0E9004E2128CDB7400F07F03128E87
:10871400FC22E56A30E10DC21B202714D227128700
:1087240065D23222C227201B07D21B128735D232D0
:108734002220520620531A02874512874512875574
:108744002290022E128CB2E0B2E7F07F04128ECE99
:10875400229004E3128CDBE0B2E7F07F04128ED99E
:108764002220520620531C028775128775128787B0
:1087740022203A2090022E128CB27400F07F041250
:108784008E4A22203B0E9004E3128CDB7400F07FAF
:1087940004128EFC22E56A30E20DC21C202814D299
:1087A400281287E8D23222C228201C07D21C128742
:1087B400B8D2322220520620531A0287C81287C820
:1087C4001287D82290022F128CB2E0B2E7F07F0514
:1087D400128ECE229004E4128CDBE0B2E7F07F0527
:1087E400128ED92220520620531C0287F81287F8D1
:1087F40012880A22203A2090022F128CB27400F0C0
:108804007F05128E4A22203B0E9004E4128CDB7406
:1088140000F07F05128EFC22E56B30E40DC21D20B2
:108824002914D22912886BD23222C229201D07D2E0
:108834001D12883BD2322220520620531A02884B42
:1088440012884B12885B22900230128CB2E0B2E79D
:0E885400F07F06128ECE229004E5128CDBE03F
:10886200B2E7F07F06128ED92220520620531C0254
:10887200887B12887B12888D22203A209002301247
:108882008CB27400F07F06128E4A22203B0E9004B6
:10889200E5128CDB7400F07F06128EFC22E56A3052
:1088A200E30DC21E202A14D22A1288EED23222C22C
:1088B2002A201E07D21E1288BED232222052062041
:1088C200531A0288CE1288CE1288DE22900231120A
:1088D2008CB2E0B2E7F07F07128ECE229004E6124D
:1088E2008CDBE0B2E7F07F07128ED92220520620FD
:1088F200531C0288FE1288FE12891022203A209010
:108902000231128CB27400F07F07128E4A22203B91
:108912000E9004E6128CDB7400F07F07128EFC22AC
:10892200E56A30E40DC21F202B14D22B128971D2BA
:108932003222C22B201F07D21F128941D23222209B
:10894200520620531A0289511289511289612290CA
:108952000232128CB2E0B2E7F07F08128ECE229081
:1089620004E7128CDBE0B2E7F07F08128ED92220F6
:10897200520620531C028981128981128993222076
:108982003A20900232128CB27400F07F08128E4AA2
:1089920022203B0E9004E7128CDB7400F07F081259
:1089A2008EFC22E56A30E50DC220202C14D22C1256
:1089B20089F4D23222C22C202007D2201289C4D2BA
:1089C200322220520620531A0289D41289D41289E3
:1089D200E422900233128CB2E0B2E7F07F09128EE9
:1089E200CE229004E8128CDBE0B2E7F07F09128E0F
:1089F200D92220520620531C028A04128A04128AA7
:108A02001622203A20900233128CB27400F07F09B1
:108A1200128E4A22203B0E9004E8128CDB7400F086
:108A22007F09128EFC22E56A30E60DC221202D1448
:108A3200D22D128A77D23222C22D202107D22112C0
:108A42008A47D2322220520620531A028A57128AA9
:108A520057128A6722900234128CB2E0B2E7F07F9A
:108A62000A128ECE229004E9128CDBE0B2E7F07F8C
:108A72000A128ED92220520620531C028A87128A99
:108A820087128A9922203A20900234128CB2740002
:108A9200F07F0A128E4A22203B0E9004E9128CDBF0
:108AA2007400F07F0A128EFC22E56A30E70DC222C2
:108AB200202E14D22E128AFAD23222C22E2022075D
:108AC200D222128ACAD2322220520620531A028A93
:108AD200DA128ADA128AEA22900235128CB2E0B2F3
:108AE200E7F07F0B128ECE229004EA128CDBE0B20A
:108AF200E7F07F0B128ED92220520620531C028BE4
:108B02000A128B0A128B1C22203A20900235128CF8
:108B1200B27400F07F0B128E4A22203B0E9004EAC0
:108B2200128CDB7400F07F0B128EFC22303221B4E7
:108B3200080A9006BE1251EDE56C04F0128B9412F5
:108B42008B5D125D111264CF1298E91299E2C23262
:108B520022128B5D125D111264CF22128B64128B72
:108B62007C2290022A128C9679007B3CE030E7014D
:108B720009A3DBF8E99002B6F0229004DF128CA47C
:108B820079007B3CE030E70109A3DBF8E990056B53
:108B9200F02220530990022A128CB2028BA6900472
:108BA200DF128CDBE020E709E550D2E1F550028BC1
:108BB200B9E550C2E1F550A3E020E709E550D2E261
:108BC200F550028BCDE550C2E2F550A3E020E70953
:0E8BD200E550D2E3F550028BE1E550C2E3F529
:108BE00050A3E020E709E550D2E4F550028BF5E50B
:108BF00050C2E4F550A3E020E709E550D2E6F55075
:108C0000028C09E550C2E6F550A3E020E709E550E3
:108C1000D2E7F550028C1DE550C2E7F550A3E020E5
:108C2000E709E551D2E0F551028C31E551C2E0F59A
:108C300051A3E020E709E551D2E1F551028C45E569
:108C400051C2E1F551A3E020E709E551D2E2F55127
:108C5000028C59E551C2E2F551A3E020E709E55144
:108C6000D2E4F551028C6DE551C2E4F551A3E02048
:108C7000E709E551D2E6F551028C81E551C2E6F5EE
:108C800051A3E020E709E551D2E7F551028C95E5C3
:108C900051C2E7F55122C3E582956CF582E58394D4
:108CA00000F58322C3E582956FF582E5839400F594
:108CB0008322128C9605A290017AE075F00CA42410
:108CC0000C05A28582378583387837F53B753C00E3
:108CD000793B12036E868208868322128CA405A239
:108CE00090017AE075F00CA4240C05A285823785EA
:108CF00083387837F53B753C00793B12036E8682EA
:108D00000886832290017CE0B40303028D1850FB97
:108D100090017EE0B4050122128D57E56B30E60329
:108D2000C23822E56A30E40630E616C2382230380E
:108D30000122D23890017AE014120AF4F0128B94D6
:108D40002230380122D23890017AE004120AF4F07D
:108D5000128D57128B942290017AE0B40009E551EC
:108D6000D2E3D2E5F55122B40109E551C2E3D2E5DF
:108D7000F55122B40209E551C2E3C2E5F55122E5FD
:108D800051D2E3C2E5F55122E56B30E603C2392248
:108D9000E56B30E403C2392230390122D239205246
:108DA0000F205306B23A128DBB22B23B128DE02245
:108DB000B23A128DBBB23B128DE022203A1BE55035
:108DC000D2E0F5504350DE4351D7129D29D232856F
:108DD0006C6D90021D7400F022E550C2E0F5502247
:108DE000203B1BE550D2E0F5504350DE4351D712F3
:108DF0009D35D232856F6E9004D27400F022E5501A
:108E0000C2E0F55022203A07E550D2E0F55022E5C5
:108E100050C2E0F55022203B07E550D2E0F5502249
:108E2000E550C2E0F55022205304128E0522128E26
:108E30001622128EC32FFF90021DE0128EA8EFF0B3
:108E400090021DE004120D77F02290021DE0FC124A
:108E50008EC32FF57C7B00900204A3E00BB57CFA57
:108E60008C7C05A2EB128EA805A2EBB57C08E57CF4
:108E70001490021DF02205A2E0A305A2F0A30B02AC
:108E80008E6A90021DE0FB900205E0256CC3956D93
:108E9000F0A3DBF6856C6D2290021DE0FB900205CD
:108EA000E0256CF0A3DBF9229002058582378583EB
:108EB000387837F53B753C00793B12036E868208A3
:108EC00086832290017AE075F00CA4240C2220E71E
:108ED00004128E4A22128E322220E704128EFC22C5
:108EE000128EE422128EC32FFF9004D2E0128F5A0A
:108EF000EFF09004D2E004120D77F0229004D2E05B
:108F0000FC128EC32FF57C7B009004B9A3E00BB557
:048F10007CFA8C7CDF
:108F140005A2EB128F5A05A2EBB57C08E57C1490F0
:108F240004D2F02205A2E0A305A2F0A30B028F1C39
:108F34009004D2E0FB9004BAE0256FC3956EF0A3D1
:108F4400DBF6856F6E229004D2E0FB9004BAE02534
:108F54006FF0A3DBF9229004BA85823785833878D1
:108F640037F53B753C00793B12036E868208868395
:108F740022753D00C200C283C2819000427439F060
:108F8400A3741DF0A37450F0A3746CF0A37479F06F
:108F9400A3740CF0A37401F0A37406F0E53DB408C7
:108FA400FB753D00D20022E53DB41023200120D200
:108FB40001C28174C0F954F053800F4280D282C23E
:108FC40082E9C454F053800F4280D282C28222E5E7
:108FD4003DB42021C2817480F954F053800F428043
:108FE400D282C282E9C454F053800F4280D282C23A
:108FF40082753D0022C201A2009281900042E58266
:10900400253DF582E0F954F053800F4280D282C2AC
:1090140082E9C454F053800F4280D282C282053D5B
:109024002212035222120352120352120352120347
:109034005212035212035212035222C28212902578
:10904400129025C281C283120352D282C287C28681
:10905400D285D284120352C282129025C281C28365
:10906400120352D282C287C286D285D2841203529C
:10907400C282129025C281C283120352D282C28755
:10908400C286D285D284120352C282129025C28132
:10909400C283120352D282C287C286D285C284128C
:1090A4000352C282129025C281C283120352D28219
:1090B400C287C286D285C284120352C2821290250C
:1090C400C281C283120352D282D287C286C285C2AF
:1090D40084120352C282129025C281C283120352A7
:1090E400D282C287C286C285C284120352C282124D
:1090F4009025C281C283120352D282D287D286D2F1
:1091040085C284120352C282129025C281C2831284
:109114000352D282C287C286C285C284120352C25B
:1091240082129025C281C283120352D282C287C2A4
:1091340086C285D284120352C282129025C281C291
:1091440083120352D282C287C286C285C2841203AA
:1091540052C282129025C281C283120352D282C2A9
:1091640087D286D285C284120352C282129025D23B
:10917400002205A2E493A305A2F0A3DBF505A22235
:10918400906D5805A29000427B20029176906D78F4
:1091940005A29000427B20029176906DC805A290B2
:1091A40000427B200291762430F02275F00A84AFCD
:1091B400F075F00A84E5F02430F0EF2430A3F022B7
:1091C40075F00A84AFF075F00A842430F0E5F024D9
:1091D40030A3F0EF2430A3F0221291C4A3742CF036
:1091E400EE2430A3F022D281C283120352D282D25F
:1091F40087D286D285D284120352C282129025D29B
:1092040081C283120352D282D287D286D285D2847B
:10921400120352C2821290252212919E12035212FC
:109224000352120352120352120352120352120334
:10923400521291847550DB7551FF1203521203527E
:109244007550CF7551FF1203521203527550DF75DA
:1092540051FE1203521203527550DF7551FB120373
:10926400521203527550DF7551BF1203521203524A
:109274007550DF75517F1203521203527550DF751A
:0E92840051EF1203521203527550DF7551FD67
:1092920012035212035275505F7551FF120352129C
:1092A200035275509F7551FF1203521203527550AB
:1092B200D77551FF1203521203527550DD7551FFDB
:1092C2001203521203527550DF7551FF12919143EE
:1092D20052FF12035212035212035212035212038A
:1092E2005212035212035212035212035212035227
:1092F2001203521203521203521203521203521257
:109302000352120352120352120352120352120355
:1093120052120352120352120352120352120352F6
:1093220012035212035212035212035253520012E8
:10933200919E12035212035212035212035222122C
:109342000352120352120352120352120352120315
:1093520052120352120352120352120352120352B6
:1093620012035212035212035212035212035212E6
:1093720003521203521203521203521203521203E5
:109382005212035212035212035212035212035286
:1093920012035212035212035212035212035212B6
:1093A20003521203521203521203521203521203B5
:1093B2005212035212035222E56B30E00122435053
:1093C20020E550C2E2F550E551C2E0F551906D98AA
:1093D20005A29000427B10129176906DA805A29092
:1093E20000527B10129176E56B30E0FBE56B30E2C8
:1093F2000630E4170293EE906DB805A29000527BFE
:109402001012917612035212959022E56B30E4FB12
:1094120012035212035222E5D220E0FBE0A305A27E
:10942200C2AF75D202F075D200D2AFA305A2DBE7BC
:1094320022E5D220E0FBC2AF75D202E075D200D2A3
:10944200AFA305A2F0A305A2DBE722900196129634
:109452002E05A27B0D90066F05A212943322900175
:10946200AD12962E05A27B0D90067C05A2129433B6
:109472002290019712969F05A27B0D90068905A264
:10948200129433229001AE12969F05A27B0D900694
:109492009605A21294332290000005A27B0D90063D
:1094A2006F05A212943390000005A27B0D90067CFA
:1094B20005A21294339000D005A27B0D9006890577
:1094C200A21294339000D005A27B0D90069605A2BD
:1094D2001294332290029E05A27B319006A605A229
:1094E200129433229002CF05A27B7C90018905A2BF
:1094F2001294332290018E12965B05A27B02900198
:109502009805A2129433229001A512965B05A27BC4
:10951200029001AF05A2129433229001B8124C6B53
:1095220012965B05A29001E9124EE37B0205A2129C
:109532009433227B0D90066F05A290000005A212C3
:109542009419227B0D90068905A29000D005A212E3
:109552009419227B319006A605A290029E05A212C2
:109562009419227B7C90018905A29002CF05A21258
:10957200941922E5D220E0FBEA930A05A2C2AF7554
:10958200D202F075D200D2AFA305A2DBE622129579
:10959200A31295B71295CB1295DF129E1C129565F8
:1095A2002290000005A27C109083C57B0D7A0012E8
:1095B2009575DCF4229000D005A27C109083DF7BAD
:1095C2000D7A00129575DCF42290029E05A27C01B0
:1095D2009083EC7B317A00129575DCF4229001A025
:1095E2007B7F79801295FAA3DBFA9001A17B7F79C8
:1095F200001295FAA3DBFA22E5D220E0FBE9C2AF22
:0E96020075D202F075D200D2AFA322E014752B
:10961000F00DA49000008582378583387837F53BBC
:10962000753C00793B12036E868208868322E0B483
:109630002B0302963950FB742BC3942B75F00DA4A9
:109640009000008582378583387837F53B753C007C
:10965000793B12036E868208868322E0C39480756C
:10966000F002A49001A08582378583387837F53BD6
:10967000753C00793B12036E868208868322E014D3
:1096800075F00DA49000D08582378583387837F542
:109690003B753C00793B12036E868208868322E08C
:1096A000B437030296AA50FB7437C3943775F00D94
:1096B000A49000D08582378583387837F53B753C98
:1096C00000793B12036E868208868322E01475F0CF
:1096D00004A49096D6739001A0229001E0229002FB
:1096E0001E2290022E2290023E2290024E229002D2
:1096F0005E2290026E2290027E2290028E2285824D
:10970000378583387837900179E01475F002A4F535
:109710003B753C00793B12036E868208868322C229
:10972000A5C2A4C295C2A3E5527F083392A6D2A3D4
:10973000C2A3DFF7B2950000C2952220360122C2F3
:10974000364350DE4351D7E550C2E0F55030521059
:10975000D23AD23B12977612982B1298E9D2322243
:1097600020530BD23A1297761298E9D23222D23B8A
:1097700012982BD23222129D2990021D7400F0857E
:109780006C6D900196E0B42B030297AE50FB1475FC
:10979000F005A4FB9079D593FA0BEB9305A21298F0
:1097A0000A05A2DAF41297D2128E98D232221294BB
:1097B0004D90066FE0FA7006129D29D23222A3E086
:1097C00005A212980A05A2DAF51297FA128E98D21B
:1097D0003222900196E01475F005A4FB9002050575
:1097E000A29079D593FAFF0BEB93240C05A2F0A37A
:1097F00005A2DAF3EF90021DF02290020505A29077
:10980000066F1298B790021DF022900236858237BB
:109810008583387837F53B753C00793B12036E86BB
:109820008208868374FFF012A09722129D3590045F
:10983000D27400F0856F6E9001ADE0B42B030298F6
:109840006350FB1475F005A4FB9079D593FA0BEBEC
:109850009305A21298C805A2DAF412987F128F4AD3
:10986000D2322212946090067CE0FAA3E005A212A4
:1098700098C805A2DAF51298A7128F4AD232229020
:1098800001ADE01475F005A4FB9004BA05A290792F
:10989000D593FAFF0BEB93240C05A2F0A305A2DAF3
:1098A000F3EF9004D2F0229004BA05A290067C1245
:1098B00098B79004D2F022E0FAFFA3E0240C05A2AE
:1098C000F0A305A2DAF4EF229004EB8582378583BA
:1098D000387837F53B753C00793B12036E86820879
:1098E000868374FFF012A097229002B6E0700122E6
:1098F000B404030298FA40FB74041475F003A490B6
:1099000099037302990F02993002995F029984902A
:1099100006D7E0FD900205E02D9006D8F0240C90CB
:1099200006D9F0240C9006DAF0240C9006DBF02225
:109930007A029006D7E0FD9006D805A2900205E0D5
:109940002DA305A2F0A305A2DAF59006D8E0240C19
:109950009006DAF09006D9E0240C9006DBF0227A2B
:10996000039006D7E0FD9006D805A2900205E02DF1
:10997000A305A2F0A305A2DAF59006D8E0240C9086
:0E99800006DBF0227A049006D7E0FD9006D8B0
:10998E0005A2900205E02DA305A2F0A305A2DAF52B
:10999E00229006D8E01206038582488583499006F8
:1099AE00D9E012060385824A85834B900195E0B477
:1099BE00020D9006DAE012060385824C85834D90E7
:1099CE0001ACE0B4020D9006DBE012060385824E78
:1099DE0085834F229002B6E0B40004129A2A22B474
:1099EE00010D129A37129ABA129B0F129B6422B46F
:1099FE00020D129A37129A8C129B0F129B6422B48C
:109A0E00030D129A37129A8C129AE1129B6422124B
:109A1E009A37129A8C129AE1129B3622129A65127A
:109A2E009ABA129B0F129B6422129A659006D8E086
:109A3E00FF900203E02490120E189006D7E02F2418
:109A4E0024C2E79006DCF0120E187464120E189001
:109A5E0006E0E0D2E0F0229006E0E020E001229065
:109A6E0006DCE0FF900203E02490120E18EF120EB7
:109A7E00187400120E189006E0E0C2E0F022129A5E
:109A8E00BA9006D9E0FF900203E02490120E1890CF
:109A9E0006D7E02F2424C2E79006DDF0120E1874CC
:109AAE0064120E189006E0E0D2E1F0229006E0E09B
:109ABE0020E101229006DDE0FF900203E0249012E7
:109ACE000E18EF120E187400120E189006E0E0C277
:109ADE00E1F022129B0F9006DAE0FF900203E024E1
:109AEE0090120E189006D7E02F2424C2E79006DEBF
:109AFE00F0120E187464120E189006E0E0D2E2F026
:109B0E00229006E0E020E201229006DEE0FF9002C5
:109B1E0003E02490120E18EF120E187400120E1895
:109B2E009006E0E0C2E2F022129B649006DBE0FFBA
:109B3E00900203E02490120E189006D7E02F2424F2
:109B4E00C2E79006DFF0120E187464120E1890061B
:109B5E00E0E0D2E3F0229006E0E020E3012290065E
:109B6E00DFE0FF900203E02490120E18EF120E18A1
:109B7E007400120E189006E0E0C2E3F022203701C6
:109B8E0022C2374350DE4351D7E550C2E0F5503084
:109B9E00520DD23AD23B129BBE129BD6D23222200B
:109BAE005308D23A129BBED23222D23B129BD622FD
:109BBE00129D2990021D7400F0856C6D129BEE12A1
:109BCE009BFF128E98D23222129D359004D27400D1
:109BDE00F0856F6E129C74129C85128F4AD23222BF
:109BEE00900197E0B43704129C262250FA129C166C
:109BFE0022900197E0B43707129C26129C552250F2
:109C0E00F7129CFA129C3B22129CFA0BEB9305A2C4
:109C1E0012980A05A2DAF422129473900689E0FAD9
:109C2E00FFA3E005A212980A05A2DAF52205A2907A
:109C3E00020505A20BEB93240C05A2F0A305A2DAF4
:109C4E00F3EF90021DF022900689E0FFFA05A29034
:109C5E00020505A2A3E0240C05A2F0A305A2DAF4E6
:109C6E00EF90021DF0229001AEE0B43704129CACCE
:109C7E002250FA129C9C229001AEE0B43707129C3F
:109C8E00AC129CDB2250F7129CFA129CC122129C41
:109C9E00FA0BEB9305A21298C805A2DAF4221294DD
:109CAE0086900696E0FAFFA3E005A21298C805A2D8
:109CBE00DAF52205A29004BA05A20BEB93240C054B
:109CCE00A2F0A305A2DAF3EF9004D2F0229006964A
:109CDE00E0FFFA05A29004BA05A2A3E0240C05A2A7
:109CEE00F0A305A2DAF4EF9004D2F022B41303022B
:0E9CFE009D025006907D98029D1FB426030221
:109D0C009D105009907E8FC39413029D1F907F85E8
:109D1C00C394261475F00DA4FB93FAFF22740079FA
:109D2C009890021EF0A3D9FC22740079989004D369
:109D3C00F0A3D9FC227908F0A3D9FC22740190017C
:109D4C00B8129D4174039001C0129D41740690019C
:109D5C00C8129D4174069001D0129D41740490016B
:109D6C00D9129D4174039001E1129D41227400901F
:109D7C000161129D41227400900151129D41227487
:109D8C0000900159129D4122740090014BF09001FA
:109D9C004CF090014EF090014FF022740090014D68
:109DAC00F0900150F0227400029DB974FF79269056
:109DBC00007AF0A3D9FC79AB9000A0F0A3D9FC22D7
:109DCC00790A9006EB7401F0A3D9FC2290066F027D
:109DDC009DE190067C74057900F07B0CA3E9F009F9
:109DEC00DBFA22900689029DF8900696740579009C
:109DFC00F07B0CA3E9F009DBFA9006A6129E132265
:109E0C009006B2129E13227B0C7401F0A3DBFC2291
:109E1C00746E900189F0740190018AF09001FFF04A
:109E2C0090018BF090019AF07411900191F07401F3
:109E3C009001A0F0900194F07402900195F07401DF
:109E4C00900192F0900193F0740390018FF07406DE
:109E5C0090019BF090019CF07404900190F07403BD
:109E6C0090019DF0740190018CF0740290018EF0C1
:109E7C00740090018DF0740090019EF004F0740158
:109E8C00900196F07401900197F074019001A1F08B
:109E9C009001A2F09001B1F074119001A8F074013E
:109EAC009001B7F09001ABF074029001ACF074012A
:109EBC009001A9F09001AAF074039001A6F0740629
:109ECC009001B2F09001B3F074049001A7F0740308
:109EDC009001B4F074019001A3F074029001A5F00C
:109EEC0074009001A4F074009001B5F004F07401BA
:109EFC009001ADF09001AEF074029001F9F0900178
:109F0C00FAF0129DD8129DDE129DEF129DF5900174
:109F1C00FB7400F09001FC7402F0C259D24F740231
:109F2C009001FDF074029001FEF09002007400F0BC
:109F3C00A37401F0A37402F0A37403F0A37409F0EA
:109F4C0022900191E014B41009C3940F7980C9C315
:109F5C00992250F575F003A4909F6873029FE30259
:109F6C009FE302A02802A02D02A03202A03702A07B
:109F7C003C02A04102A04602A04B029FE3029FEBD1
:109F8C00029FF3029FFD02A00502A0119001A8E020
:109F9C0014B41009C3940F7980C9C3992250F57574
:109FAC00F003A4909FB373029FE3029FE302A050BF
:109FBC0002A05502A05A02A05F02A06402A069028E
:109FCC00A06E02A073029FE3029FEB029FF3029F1D
:109FDC00FD02A00502A011126C00547FD2E02212E7
:109FEC006C00543F244022126C0075F00584244C04
:109FFC0022126C00541F246022126C00541F75F046
:10A00C000284247022126C0054016008126C0054FB
:10A01C001F245422126C00540F247022740202A0CC
:10A02C0078740302A078740402A078740502A078F6
:10A03C00740602A078740702A078740802A07874E1
:10A04C000902A078740202A07F740302A07F74043A
:10A05C0002A07F740502A07F740602A07F74070221
:10A06C00A07F740802A07F740902A07F90019EF06B
:0EA07C0002A0839001B5F0F57CA3E004B57C52
:10A08A00067400F0747F2250F8F074642222F9906A
:10A09A000041E0B400012290003FE0900000F58208
:10A0AA00E9F090003FE004B43F027400F0900041F0
:10A0BA00E014F022C2AC900041E0B43E03D2AC22DC
:10A0CA0004F0900040E0900000F582E0F990004032
:10A0DA00E004B43F027400F0D2ACE9120E5202A0BE
:10A0EA00BE304ED0C24E2212A0FB12A12A12A1519A
:10A0FA00229001FBE030E00122C2AD1204B8D2ADD9
:10A10A0012045C75F00A8404120BB9F57C9006E21D
:10A11A00E0B57C0122E57CF090018AF0128B532293
:10A12A00C2AD1204ACD2AD12045C75F03F840412C5
:10A13A000CB9F57C9006E3E0B57C0122E57CF09051
:10A14A00018CF0128B53229006E8E01475F003A4F8
:10A15A0090A15E7302A1D202A20702A22702A24222
:10A16A0002A26402A27102A27E02A28B02A2A80229
:10A17A00A2CF02A2DB02A2F902A31E02A32B02A310
:10A18A003802A34502A36202A38002A3A502A3B2D6
:10A19A0002A3BF02A3CC02A3E902A40702A42C02D1
:10A1AA00A43902A44602A45302A47002A48E02A4F3
:10A1BA00B302A4C002A4CD02A4DA02A1EEC2AD1277
:10A1CA0004A0D2AD12045C2212A1C775F002841257
:10A1DA000C05F57C9006E6E0B57C0122E57CF09062
:10A1EA00018DF02212A1C7120A4C14F57C9006E6E2
:10A1FA00E0B57C0122E57CF0900189F02212A1C72A
:10A20A0075F01C8404120BDFF57C9006E6E0B57C41
:10A21A000122E57CF090018BF0128B532212A1C728
:10A22A00F57C9006E6E0B57C0122E57CF090018E93
:10A23A00F01232041231222212A1C775F00F8404DF
:10A24A00120CA6F57C9006E6E0B57C0122E57CF0CE
:10A25A0090018FF01232C9D2492212A1C775F03388
:10A26A008404240102A24D12A1C775F03384042488
:10A27A000702A24D12A1C775F0408404240D02A260
:10A28A004D12A1C775F0188404120CCCF57C900607
:10A29A00E6E0B57C0122E57CF0900190F02212A163
:10A2AA00C775F0028404120AE1797FC9C39924119F
:10A2BA00120C15F57C9006E6E0B57C0122E57CF0EF
:10A2CA00900191F02212A1C775F01284240302A210
:10A2DA00BD12A1C7F57C9006E6E0B57C0122E57CBB
:10A2EA00F09001B8F090017D7401F0124DFD221238
:10A2FA00A1C775F00F8404120CA6F57C9006E6E05F
:10A30A00B57C0122E57CF09001C0F079019001D87A
:10A31A00E049F02212A1C775F0338404240102A394
:10A32A000412A1C775F0338404240702A30412A1FE
:10A33A00C775F0408404240D02A30412A1C775F066
:10A34A00188404120CCCF57C9006E6E0B57C012258
:10A35A00E57CF09001D9F02212A1C7F57C9006E6BF
:10A36A00E0B57C0122E57CF09001B9F090017D74A2
:10A37A0002F0124DFD2212A1C775F00F8404120CCF
:10A38A00A6F57C9006E6E0B57C0122E57CF090011A
:10A39A00C1F079029001D8E049F02212A1C775F004
:10A3AA00338404240102A38B12A1C775F0338404F9
:10A3BA00240702A38B12A1C775F0408404240D025E
:10A3CA00A38B12A1C775F01884F57C9006E6E0B558
:10A3DA007C0122E57C04120CCCF09001DAF0221206
:10A3EA00A1C7F57C9006E6E0B57C0122E57CF090F9
:0EA3FA0001BAF090017D7403F0124DFD2212A5
:10A40800A1C775F00F8404120CA6F57C9006E6E04F
:10A41800B57C0122E57CF09001C2F079049001D866
:10A42800E049F02212A1C775F0338404240102A484
:10A438001212A1C775F0338404240702A41212A1D2
:10A44800C775F0408404240D02A41212A1C775F048
:10A45800188404120CCCF57C9006E6E0B57C012249
:10A46800E57CF09001DBF02212A1C7F57C9006E6AE
:10A47800E0B57C0122E57CF09001BBF090017D7491
:10A4880004F0124DFD2212A1C775F00F8404120CBE
:10A49800A6F57C9006E6E0B57C0122E57CF090010B
:10A4A800C3F079089001D8E049F02212A1C775F0ED
:10A4B800338404240102A49912A1C775F0338404DB
:10A4C800240702A49912A1C775F0408404240D0240
:10A4D800A49912A1C775F0188404120CCCF57C90CD
:10A4E80006E6E0B57C0122E57CF09001DCF0221262
:10A4F800A50112A53312A55A22C2AD1204D0D2ADBD
:10A5080012045C75F00A8404120BB9F57C9006E419
:10A51800E0B57C0122E57CF09001A1F09001FBE020
:10A5280030E00412A9B522128B5322C2AD12049452
:10A53800D2AD12045C75F03F84F57C9006E5E0B579
:10A548007C0122E57C04120CB9F09001A3F0128B77
:10A5580053229006E9E01475F003A490A5677302EE
:10A56800A5D802A5F402A61402A62F02A65102A697
:10A578005E02A66B02A67802A69502A6BC02A6C831
:10A5880002A6E602A70B02A71802A72502A7320215
:10A59800A74F02A76D02A79202A79F02A7AC02A726
:10A5A800B902A7D602A7F402A81902A82602A8335E
:10A5B80002A84002A85D02A87B02A8A002A8AD02DA
:10A5C800A8BA02A8C7C2AD1204C4D2AD12045C2254
:10A5D80012A5CD75F00284120C05F57C9006E7E013
:10A5E800B57C0122E57CF09001A4F02212A5CD757E
:10A5F800F01C8404120BDFF57C9006E7E0B57C01C3
:10A6080022E57CF09001A2F0128B532212A5CDF521
:10A618007C9006E7E0B57C0122E57CF09001A5F08E
:10A62800123C21123BAE2212A5CD75F00F84041204
:10A638000CA6F57C9006E7E0B57C0122E57CF0905D
:10A6480001A6F0123C79D24A2212A5CD75F03384C6
:10A6580004240102A63A12A5CD75F0338404240718
:10A6680002A63A12A5CD75F0408404240D02A63A3C
:10A6780012A5CD75F0188404120CCCF57C9006E771
:10A68800E0B57C0122E57CF09001A7F02212A5CD6F
:10A6980075F0028404120AE1797FC9C39924111262
:10A6A8000C15F57C9006E7E0B57C0122E57CF0907E
:10A6B80001A8F02212A5CD75F01284240302A6AADF
:10A6C80012A5CDF57C9006E7E0B57C0122E57CF08B
:10A6D8009001BCF090017D7405F0124DFD2212A589
:10A6E800CD75F00F8404120CA6F57C9006E7E0B552
:10A6F8007C0122E57CF09001C4F079109001D8E04B
:10A7080049F02212A5CD75F0338404240102A6F184
:10A7180012A5CD75F0338404240702A6F112A5CD45
:10A7280075F0408404240D02A6F112A5CD75F01829
:10A738008404120CCCF57C9006E7E0B57C0122E598
:10A748007CF09001DDF02212A5CDF57C9006E7E0C3
:10A75800B57C0122E57CF09001BDF090017D740686
:10A76800F0124DFD2212A5CD75F00F8404120CA62F
:0EA77800F57C9006E7E0B57C0122E57CF090D0
:10A7860001C5F079209001D8E049F02212A5CD75D7
:10A79600F0338404240102A77812A5CD75F0338422
:10A7A60004240702A77812A5CD75F0408404240D71
:10A7B60002A77812A5CD75F0188404120CCCF57C8E
:10A7C6009006E7E0B57C0122E57CF09001DEF02200
:10A7D60012A5CDF57C9006E7E0B57C0122E57CF07C
:10A7E6009001BEF090017D7407F0124DFD2212A576
:10A7F600CD75F00F8404120CA6F57C9006E7E0B543
:10A806007C0122E57CF09001C6F079409001D8E009
:10A8160049F02212A5CD75F0338404240102A7FF66
:10A8260012A5CD75F0338404240702A7FF12A5CD27
:10A8360075F0408404240D02A7FF12A5CD75F0180B
:10A846008404120CCCF57C9006E7E0B57C0122E589
:10A856007CF09001DFF02212A5CDF57C9006E7E0B2
:10A86600B57C0122E57CF09001BFF090017D740873
:10A87600F0124DFD2212A5CD75F00F8404120CA620
:10A88600F57C9006E7E0B57C0122E57CF09001C7F7
:10A89600F079809001D8E049F02212A5CD75F03309
:10A8A6008404240102A88612A5CD75F033840424FD
:10A8B6000702A88612A5CD75F0408404240D02A8CF
:10A8C6008612A5CD75F0188404120CCCF57C900682
:10A8D600E7E0B57C0122E57CF09001E0F02212A8C9
:10A8E600EE12A9101298E922C2AD1204E8D2AD12F6
:10A8F600045C75F01584F57C9006D7E0B57C0122E2
:10A90600E57CF01298E91299E222C2AD1204DCD27B
:10A91600AD12045C75F0178404F57C9006E1E0B591
:10A926007C0122E57CF0F57C9006D6E0B57C0F90A4
:10A936000185E57CF0D2571298E91299E22250EF90
:10A94600229001FDE0B404012212135D9006A5E0F9
:10A9560020E2012220E50122C2E2C2E5F09001FBDD
:10A96600E0B2E0F020E00412A9D12212A9AD2290B3
:10A9760001FBE020E00412A9D12212A98422C2918F
:10A986009001A1E0B4190302A99820E0041402A9D9
:10A99600980490018AF0128B53229001FBE020E08C
:10A9A60003D29122C2912290018AE09001FFF0C267
:10A9B600919001A1E0B4190302A9C920E004140290
:10A9C600A9C90490018AF0128B5322D2919001FFFB
:10A9D600E090018AF0128B532243B71843B81275E0
:10A9E6008790758922758DF8758BF8D28E7598507B
:10A9F600C299C298D2ACC2117553287554047555C4
:10AA06007D75560290FF9C8582CA8583CB8582CC54
:10AA16008583CD43C804D2ADD2AF2243B74043B8F5
:10AA2600408541EA8542FA43D90143DA4975570818
:10AA360075580CD2DED2AE22C0E0C0D030DF07C2DD
:10AA4600DFD0D0D0E032C2D8E5EA2541F5EAE5FA12
:10AA56003542F5FAD5570B755708D209D5580375FF
:10AA6600580CD0D0D0E032C0E0C0D0E582C0E0E5DE
:10AA760083C0E0C2D4D2D3309911C211C299D0E0BA
:10AA8600F583D0E0F582D0D0D0E032309807C29876
:10AA9600E59912A098D0E0F583D0E0F582D0D0D029
:10AAA600E032C0E0C0D0E582C0E0E583C0E0D2D4A9
:10AAB600C2D3C2CF201212D55D0F755DFFD55E09D8
:10AAC600855B5D855C5E12227E201312D5630F7551
:10AAD60063FFD5640985616385626412257DD5535C
:10AAE6003B7553281204F4128FAB12063312064438
:0EAAF60012971FD55426755406128496B21678
:10AB040012845DD55518755532C205900176E06002
:10AB14000214F0D55608755603D205126C4AD0E0DB
:0BAB2400F583D0E0F582D0D0D0E03205
:00000001FF
